:10000000026F740270980000000000026C82000011
:100010000000000270BF000000000032000000007D
:10002000000000023DE80000000000026D7B0000BF
:1000300074A21200C4E81200FFE91200FF12013698
:100040002274A21200C4E81200FFE71200FF09D5D3
:1000500082F81201362274A21200C4E81200FF7462
:10006000A31200C412011FF709D58204120136221F
:10007000C296D297000000C29780E974A21200C411
:10008000E81200FF1200882274A31200C412011F9C
:10009000F91201362274A27A08C296000000C297B3
:1000A000335005D2960200AAC296D297000000C231
:1000B00097DAEDD29600D297000000309604C297EE
:1000C000C322D3227A08D296D29700000000000003
:1000D00000000000000000000000C296000000C206
:1000E00097335005D2960200EBC296D297000000DB
:1000F000C297DAEDD29600D297000000C297227A1A
:1001000008335005D29602010BC296D29700000028
:10011000C297DAEDD29600D297000000C297227AF9
:1001200008D296C29700000000D297C3309601B360
:1001300033DAF0C29722C296000000D29700000086
:10014000D2962278767600087600787AE6543FF6E2
:1001500078007976C082758207120041D08212063B
:10016000522278027978C082758205120056D082B8
:1001700022787CE603C4540775F018A4C0E0787AAE
:10018000E6C4540375F00AA4F5F0E6540F25F0D048
:10019000F025F075F03CA4C0F0C0E07879E6C454D6
:1001A0000775F00AA4F5F0E6540F25F0D0F025F01D
:1001B000F5F0D0E03400C5F02250523430322076D1
:1001C00065722E3131392E30204864773A48203418
:1001D000303030752033312D30382D3034203131EE
:1001E0003A34392020284329526F676572205370B2
:1001F0002E4A2E207777772E726F6765722E706C7D
:100200002C2074656C2F666178202B3438203535AE
:100210002032373230313332202843296A502D7052
:100220006C2C204D6F6E61204C6973612043452C0E
:100230002049534F393030312C2031737420436CB6
:10024000617373D320202052204520532045205431
:10025000D25052333032204C434420763131392E43
:1002600030002D2D2F2D2D202D2D3A2D2D004350DA
:10027000523A20004C6F633A20004C4F433A200022
:10028000D2202020202020202020202020202020BC
:1002900020D200454E545259202020004558495440
:1002A00020202020004455545920455849540049E5
:1002B0004E5445524E414C00D12020202020202079
:1002C000202020202020202020D143524320202005
:1002D000204520722072206F2072002020202020D4
:1002E0000020D1466C6173682043524320457272EE
:1002F0006F722000D3436F6E666967204D656D2075
:100300004572726F7200D3205365727669636520FF
:100310004F4E00D32053657276696365204F464681
:1003200000D2204D4153544552204944203D2020C5
:100330003F2000D35365742074696D652048484D93
:100340004D202020D200D353657420646174652051
:10035000524D4D44445720D200D22020202020204E
:1003600020202020202020202020D2D50105524509
:10037000473A200000D3D5021044206F2077206E2A
:10038000206C206F206120642000D12020202020BC
:10039000202020202020202020202020D1D5030C28
:1003A00050617373776F72643F203A2000D2D50496
:1003B00010204163636573732064656E6965642012
:1003C0002000D2D5051020416363657373206772E6
:1003D000616E7465642000D1D504102041636365AB
:1003E00073732064656E6965642020D2D506102081
:1003F0004E6F204475616C20456E74727920200028
:10040000D3D509104475616C20456E747279204D06
:100410006F64652000D1D50A0A2020204572726FD2
:10042000722023002020202000D1D50C1020202075
:100430004150422052657365742020202000D2D59F
:100440000E104C696D697420657863656564656438
:10045000202000D50F0C4E4F524D414C2020202023
:10046000202000D1D5041020204143434553532080
:1004700044454E59202020D2D51010204150422012
:1004800056696F6C6174696F6E202000D1D50D10B4
:10049000202020204964656E74204F4B20202020AE
:1004A000D2D51010204150422056696F6C6174699A
:1004B0006F6E202000D2D51110204E6F206F6E6518
:1004C00020696E73696465202000D1D51210202048
:1004D0002055736572204944203D203F202000D3E1
:1004E0002020202055205320452052D2D516102000
:1004F0002050726F6772616D6D696E6700D3202046
:1005000020494E5354414C4C455220202020D2D5F6
:100510001610202050726F6772616D6D696E6720D2
:10052000202000D220202020462052204520452097
:100530002020202000D22020204520582049205370
:1005400020542053202000D1D504102020414343C3
:100550004553532044454E59202020D2D506102023
:1005600020496E70757420426C6F636B732020009D
:10057000D1D5041020204143434553532044454ED8
:1005800059202020D2D507102020434C4F534544FA
:10059000204D4F444520202000D1D504102020417B
:1005A00043434553532044454E59202020D2D5087B
:1005B000104F7574206F662074696D65207A6F6EB8
:1005C0006500D1D5041020204143434553532044B6
:1005D000454E59202020D2D50B10204F464620638F
:1005E0006F6E646974696F6E202000D1D51310207E
:1005F000205357495443482044454E59202020D287
:10060000D508104F7574206F662074696D65207A67
:100610006F6E6500D1D504102020414343455353EC
:100620002044454E59202020D2D5141020202020CF
:10063000505245414C41524D2020202000D1D5152B
:10064000102053776974636865722049443D203FE8
:100650002000C28E53890F438910758BD6758D97F4
:10066000C28FD28E308FFDC28E22C28E53890F432D
:100670008910758BEB758DCBC28FD28E308FFDC2FA
:100680008E22C28E53890F438910E58AC4242BF52C
:100690008B758DEBC28FD28E308FFDC28E22F9C347
:1006A000137004A24D801814C0E0030303540F24F8
:1006B0007CF8D0E0540704F5F0E213D5F0FCE992A1
:1006C000E02275F00612077922C2A075F006120723
:1006D00079D2A0221206C91206C21206C91206C297
:1006E0001206C91206C21206C91206C21206C9753E
:1006F000F01812077922C2A075F04B120779D2A028
:1007000022755104123B19C2A075F0C8120779D2A4
:10071000A022755105123B191206F675F01E12073C
:10072000791206F622755107123B191206E022755E
:100730005106123B191206E6221206D41206D422E2
:10074000755107123B19755106123B191206E61234
:1007500006E61206E6221206E61206DA22C2A1C256
:10076000621206C975F012120779D2A1C262221272
:1007700006C975F01212077922120652201507C019
:10078000F0122BA9D0F0D5F0F0227004A24DB322C4
:10079000C0E014120799D0E022C0E0030303540F15
:1007A00028F8D0E0C0E0540704F5F0E213D5F0FCDF
:1007B000D0E0221206D475F064120652D5F0FA2267
:1007C0001206E075F0C8120652D5F0FA80F222E562
:1007D00073B400030208C4B40717C2AC1206821235
:1007E0000682D299120987C259D2B6126D860208C2
:1007F000C1B40117C2AC120682120682D299121538
:10080000CDC259D2B6126D860208C1B40317C2AC6C
:10081000120682120682D299121652C259D2B6120A
:100820006D860208C1B40217C2AC1206821206829B
:10083000D2991214EEC259D2B6126D860208C1B412
:100840000417C2AC120682120682D299121530C267
:1008500059D2B6126D860208C1B40517C2AC120691
:1008600082120682D2991208F0C259D2B6126D864F
:100870000208C1B40617C2AC120682120682D299CF
:1008800012169AC259D2B6126D860208C1B4081760
:10089000C2AC120682120682D299126989C259D25A
:1008A000B6126D860208C1B40917C2AC12068212D4
:1008B0000682D299126A16C259D2B6126D86020801
:1008C000C1757300E56E6013B40105122FE980084D
:1008D000B40205122FF88000756E00122BA9304566
:1008E0000B20A808305F05C25F1230251268542221
:1008F000C2B61201627537007403124DA4E51E12D0
:100900004DA4E51F124DA47457124DA4787BE62325
:10091000235403124DA4787CE630E402240A540FD9
:10092000124DA4787BE6C4540375F00AA4F5F0E6F2
:10093000540F25F0124DA4787AE6C4540375F00ADA
:10094000A4F5F0E6540F25F0124DA47879E6C454CE
:100950000775F00AA4F5F0E6540F25F0124DA478BF
:1009600078E6C4540775F00AA4F5F0E6540F25F0B4
:10097000124DA4787CE603C45407124DA4E5371247
:100980004DA43099FDD322126BD8C2B675370074CE
:1009900003124DA4E51E124DA4E51F124DA4745080
:1009A000124DA4747D124DA4900000E535600F90A7
:1009B00003E81460099007D0146003900BB87E7DA3
:1009C0007F0875F000C0F0126BD3B40203D380012E
:1009D000C3D0E033F5F0A3DFEC124DA4DEE2E5373F
:1009E000124DA43099FD22C0F075F0DCD5F005B2AF
:1009F000B51264F7C0F0120C31D0F030E7EED0F051
:100A000022AAF01209E7E532652FF5F0E5336530EB
:100A100045F0600C120B58852F328530331209E7F0
:100A2000120BF61209E7120C1E1209E7120B658A67
:100A3000F022AAF01209E7E532652FF5F0E53365FB
:100A40003045F0600C120B58852F32853033120977
:100A5000E7120BE21209E7120C1E1209E7120B65EE
:100A60008AF0227920752F017530037531E09000EE
:100A7000BA1209E7120B581209E7120BB679007582
:100A80002F017530047531009000DA1209E7120B5E
:100A9000581209E7120BB679E0752F01753005750C
:100AA00031009001DA1209E7120B581209E7120B14
:100AB000B6852F3285303322AAF01209E7E5326578
:100AC0002FF5F0E533653045F0600C120B58852F9B
:100AD000328530331209E7120B9E8AF022AAF012F7
:100AE00009E7E532652FF5F0E533653045F0600C38
:100AF000120B58852F328530331209E7120B868A84
:100B0000F022C0F075F00833C297928300D297D5D7
:100B1000F0F5D0F022C0F075F008C297D29700A28D
:100B20008233D5F0F5D0F022D2B7D297D283D282D9
:100B3000D28422E53033E52F3322C3E5303322E57A
:100B40003122120B02120B33120B02120B3A120B50
:100B500002120B3F120B0222120B28C28474531292
:100B60000B42D28422120B28C2847458120B42D238
:100B70008422120B28C2847454120B42E4120B021A
:100B8000120B15D28422120B28C2847454120B4209
:100B9000E4120B02120B15F608D9F9D28422120BBB
:100BA00028C2847454120B42E4120B02120B15F289
:100BB00008D9F9D28422120B28C2847454120B4231
:100BC000E4120B02120B15F0A3D9F9D28422120BF6
:100BD00028C0E0C2847484120B42D0E0120B02D20F
:100BE0008422120B28C2847484120B42E6120B0278
:100BF00008D9F9D28422120B28C2847484120B42C1
:100C0000E2120B0208D9F9D28422120B28C2847492
:100C100084120B42E0120B02A3D9F9D28422120BE8
:100C200028C2847483120B42D284120652120652D6
:100C300022C2847457120B02120B15D28422D28363
:100C4000D282D297D2B7D284B2B575F002120652D0
:100C5000D5F0FAC2B7B2B575F002120652D5F0FA65
:100C6000D2B7B2B522752F017530DB75310012098C
:100C7000E7120F007532FF7533FF22AE83AD82900D
:100C8000DB007F207404F97476F8752F01858330BA
:100C9000858231120ADD7876E66E702508E66D7081
:100CA0002008E6601AB4FF028013167404F9747603
:100CB000F8752F01858330858231120A32C322D321
:100CC00022A3A3A3A3DFBD80F490DB007F207404E4
:100CD000F97476F8752F01858330858231120ADD2B
:100CE0007876E66E700908E66D700408E6FC22A3CB
:100CF000A3A3A3DF0A7CFF2290DB007F207BFF748D
:100D000004F97476F8752F01858330858231120AD3
:100D1000DD7876E66E702C08E66D702708ECB4FF7F
:100D20000D787676FF0876FF0876FF0874FFF67474
:100D300004F97476F8752F01858330858231120AA3
:100D400032C322BBFF107876E6B4FF0A08E6B4FF90
:100D500005C374209FFBA3A3A3A3DFA3BBFF02D300
:100D600022EB232354FC2400F5827583DB5002051B
:100D7000837876EEF608EDF608ECF608E4F67404EF
:100D8000F97476F8752F01858330858231120A3225
:100D9000C32275830075F08E752F028583307531FF
:100DA00000C0F0C0831209E7120F00D0830583D082
:100DB000F0D5F0E475830075F0DA752F0385833084
:100DC000753100C0F0C0831209E7120F00D083050F
:100DD00083D0F0D5F0E47532FF7533FF22758300C0
:100DE00075820075F08EC0F0C082C083752F0285B9
:100DF00083307531001209E7120B58D083D082C0BE
:100E000082C083752F008582307531001209E71288
:100E10000C1ED083D08205830582D0F0D5F0C77533
:100E2000830075820075F0DAC0F0C082C083752F30
:100E3000038583307531001209E7120B58D083D037
:100E400082C082C083752F018582307531001209FE
:100E5000E7120C1ED083D08205830582D0F0D5F036
:100E6000C77532FF7533FF2275830075820075F0F8
:100E70008EC0F0C082C083752F008583307531002D
:100E80001209E7120B58D083D082C082C083752F1D
:100E9000028582307531001209E7120C1ED083D012
:100EA0008205830582D0F0D5F0C775830075820076
:100EB00075F0DAC0F0C082C083752F01858330756C
:100EC00031001209E7120B58D083D082C082C08350
:100ED000752F038582307531001209E7120C1ED080
:100EE00083D08205830582D0F0D5F0C77532FF75B7
:100EF00033FF22120B28C2847450120B42D2842278
:100F0000120B28C2847481120B42D28422120B2845
:100F1000C2847484120B42E8120B02D9FAD28422E2
:100F2000AAF01209E7E532652FF5F0E533653045A3
:100F3000F0600C120B58852F328530331209E712FE
:100F40000F0D1209E7120C1E8AF022120B28C28420
:100F50007454120B42E4120B02E4C0E0120B15D0E1
:100F6000F025F0D9F5D284227583007582028006BF
:100F7000758300758200E475F08D85822F8583303E
:100F8000753100C082C083C0F0C0E01209E7120BC7
:100F9000581209E77900120F4BD0F025F0D0F0D0AD
:100FA00083D0820583D5F0D285822F858330753139
:100FB00000C0E01209E7120B581209E77920120F5E
:100FC0004BD0F025F07532FF7533FF227583007525
:100FD00082038006758300758201E475F0DA8582EC
:100FE0002F858330753100C082C083C0F0C0E0120D
:100FF00009E7120B581209E77900120F4BD0F025C0
:10100000F0D0F0D083D0820583D5F0D27532FF7551
:1010100033FF05E02275830075F000752F0085838E
:1010200030753100C0F0C0831209E7120F00D08381
:101030000583D0F0D5F0E47532FF7533FF7583007A
:1010400075F0DA752F01858330753100C0F0C083EB
:101050001209E7120F00D0830583D0F0D5F0E475B4
:1010600032FF7533FF221206EC754BFA3090FA7599
:10107000F005120652D5F0FA754BFA2090FA2222AA
:1010800022222222300759787BE6540FC0E0E6C4C2
:10109000540375F00AA4D0F025F0FD787CE630E426
:1010A00002240A540FFE901A007F3C7404F9740065
:1010B000F8752F01858330858231120AB87800E2F5
:1010C0006D701708E26E701208E2C42354E0F5F068
:1010D000787CE6541F45F0F68006A3A3A3A3DFCBDC
:1010E00022120162121084120171FEAFF0126644E6
:1010F0007DFF0DED30E70122D26D75F004A424BA16
:10110000F582E5F03400F583C082C0837876E0F69E
:10111000A308E0F6A308E0F6A308E0F6D083D082A7
:10112000121081787686830886827876B6FF070863
:10113000B6FF0302119AC3E58233F582E58333F5E6
:1011400083E58224E0F582E5833405F5837878E64B
:10115000704808E66044FB7402F97476F8752F0154
:10116000858330858231120ADD121082A3A378763E
:10117000E60856B4FF0302119A787686F053F07FA2
:1011800008E6C39EC0E0E5F09FD0F0400445F07053
:10119000097876E6A2E7926DDBBD121083BD003DB3
:1011A000B26D122F6E403320303020160E30310BCE
:1011B000204C05306D248003206D1FA26D924C924F
:1011C000E0A24D92E1F5F013924D65F030E00B2076
:1011D0004D0512300780031230160210F2ED14C0D4
:1011E000E0030303540F247CF8D0E0540704FB749D
:1011F00000D333DBFD306D05FBE24B8004F4FBE2F2
:101200005BF20210F2120B02120B33120B02120BE2
:101210003AD2E0120B02120B3F120B0222120B28E1
:10122000C2847454121205E4120B02120B15F60854
:10123000D9F9D28422120B28C2847484121205E6D2
:10124000120B0208D9F9D2842290FC00752F047584
:101250003000753100C082C083754BFA1209E71265
:101260000B58852F6D85306C790878761209E71256
:10127000121D121445D083D0827044C082C083787E
:101280007A86830886821212F6402478788683084C
:1012900086821212F64018121315E582600AE56A7A
:1012A000B56C0CE56BB56D07D083D0820212D17896
:1012B00078E6249AF61214881261B4D083D082059D
:1012C00030E5307002052FA3E58245837087121246
:1012D000D87532FF7533FF2278787600087600786B
:1012E0007A7600087600087600087600756D047539
:1012F0006C0012146422C082C083E5822400F5824F
:10130000E5833480F5834005D083D08222D083D01A
:101310008290000022E58275F008A4F582E5F0C510
:101320008375F008A42583F583E5F03404F56BE5B7
:10133000822400F582E5833400F5835002056B8535
:10134000836A221261C4D083D08222C082C08312F9
:10135000141E70EF787886830886821212F640E3B6
:101360001213151216FF78767600787AE518F608CB
:10137000E519F60876000876007408F97476F885A1
:101380006B2F858330858231120A327404F9747AA6
:10139000F8856B2F858330858231120ADD75F00464
:1013A0007876797AE667600280990809D5F0F512B7
:1013B000142578788683088682A31212F67878A698
:1013C0008308A682787A86830886821212F6787855
:1013D000E66583700A08E665827004A31212F67847
:1013E0007AA68308A682C06DC06C856B6D856A6C19
:1013F000121464D0E0D0F0B56C09C5F0B56D028070
:1014000018C5F0C06DC06C85F06DF56C7878E62479
:1014100099F6121488D06CD06DD083D08222121429
:101420002512144522856D2F856C30753100120907
:10143000E7120B58790878761209E712121D852FEA
:101440003285303322787BE6182618261826182491
:101450005566700F787BE618661866186618661869
:101460006499662212146B12148822787BE618267F
:1014700018261826182455F6787BE618661866187C
:10148000661866186499F622856D2F856C30753163
:10149000001209E7120B581209E779087876121240
:1014A000351209E7120C1E1209E7120B65852F325F
:1014B0008530332212141E70307878E6C0E008E6DA
:1014C000C0E0088683088682C3D0E09582F582D08A
:1014D000E09583F58350104582600CE5822400F589
:1014E00082E5833480F583C322900000D322C2B604
:1014F0001214B4E433C0E07537007403124DA4E550
:101500001E124DA4E51F124DA47453124DA4D0E039
:10151000124DA47400124DA47400124DA4E5831260
:101520004DA4E582124DA4E537124DA43099FD2259
:10153000C2B6E5356004F4FF8004FF1212D8753797
:10154000007403124DA4E51E124DA4E51F124DA414
:101550007456124DA4EF124DA4E537124DA43099E4
:10156000FD227401C0E0787675F008E4F608D5F045
:10157000FBD0E0D3221214B440E860E8787A868386
:10158000088682121588C322C082C083E58275F066
:1015900008A4F582E5F0C58375F008A42583F583DA
:1015A000E5F03404F56BE5822400F582E583340030
:1015B000F5835002056B7408F97476F8856B2F85F6
:1015C0008330858231120ADDD083D082221214B496
:1015D0007F0850051212D87F007878865A08865BFB
:1015E00008865C08865DC2B67537007403124DA488
:1015F000E51E124DA4E51F124DA47454124DA4E52E
:1016000035124DA4EF124DA4E535603CE55D655BF8
:10161000F5F0E55C655A45F0600B855D82855C837D
:101620001215888003121564855D82855C83A31280
:1016300012F685825D85835C787675F008E6124D3A
:10164000A408D5F0F8D535C4E537124DA43099FD7E
:10165000C322E5357007C2AF1214B45005E535F466
:10166000800C787AA65C08A65D121464E535D2AFCA
:10167000C0E0C2B67537007403124DA4E51E124DCA
:10168000A4E51F124DA47455124DA4D0E0124DA430
:10169000E537124DA43099FDD322C2B675370074D8
:1016A00003124DA4E51E124DA4E51F124DA474585B
:1016B000124DA47420232354FC04124DA474201250
:1016C0004DA490DB007F207404F97476F8752F0127
:1016D000858330858231120ADD7876E6124DA408C2
:1016E000E6124DA408E6124DA408E6124DA408A384
:1016F000A3A3A3DFD2E537124DA43099FDD3221264
:101700000162787CE630E402240A540FC4F9787B45
:10171000E6C4540375F00AA4F5F0E6540F25F0C3AF
:1017200013497877F6787BE692E754C0F97879E642
:10173000C4540775F00AA4F5F0E6540F25F049F9F2
:10174000787AE6C4540375F00AA4F5F0E6540F2540
:10175000F0F5F07878E654702345F07879F67878EB
:10176000E9F622C082C083E52F12620EE5301262D4
:101770000E7878E612620E08E612620E08E6126231
:101780000E08E612620E121066D083D082225359E0
:101790000F53580F5318F053190FC2AFE5582324B5
:1017A000A7F8E5184519F608A61A055853580FE585
:1017B00058B55905055953590FD2AFC3E558955936
:1017C0005002241024F4500375630022E559B558E3
:1017D000057400780022C33324A7F8E6C0E008E6C9
:1017E000F8D0E02222304EFDC2A075F00612077933
:1017F000D2A075F014120779E53FC24E22301503CE
:10180000754AF0122555204E07740F30150580F3E8
:101810001217E522C226A226B392A522D226A2261C
:10182000B392A522B226A226B392A522F5F0030315
:10183000543FB4025BE53864086005E538B40D4DEB
:10184000E5F089F0C0F030071CC0E078B0E260132A
:10185000C3335005D0E002187412069E50F6D0E053
:10186000021865D0E0D0F0A9F05403B4020D1218AC
:101870001402195FD0F0A9F002195FB40106121822
:101880001C02195FB4030612182402195F02195DC5
:10189000B40365E53964086005E539B40DEFE5F09A
:1018A00089F0C0F030071CC0E078B1E26013C333A8
:1018B0005005D0E00218D612069E50F6D0E002186D
:1018C000C3D0E0D0F0A9F05403B40211C227A2277C
:1018D000B392A602195FD0F0A9F002195FB4010A11
:1018E000D227A227B392A602195FB40309B227A296
:1018F00027B392A680698065B40462E53A64086003
:1019000005E53AB40D57E5F089F0C0F030071CC08A
:10191000E078B7E26013C3335005D0E002193D12FE
:10192000069E50F6D0E002192BD0E0D0F0A9F0547A
:1019300003B4020FC22BA22BB392808022D0F0A955
:10194000F0801CB40109D22BA22BB392808010B47A
:101950000309B22BA22BB3928080048000D322C350
:101960002278AC75F00EE4F208D5F0FB74FF78B481
:10197000F278B5F222D24E6F20657874656E646598
:10198000642020202020202020007564FF1219618F
:10199000C207C206120FD4704F120A637401F974A1
:1019A00064F8752F017530037531A0120ADD740ECD
:1019B000F974ACF8752F017530037531A1120AB8AE
:1019C0007410F9748CF8752F017530037531C012DD
:1019D0000AB87410F9749CF8752F017530037531CD
:1019E000D0120AB8D207D2062222E8C0E07869E213
:1019F000F572D0E0F822E8C0E0786AE2F572D0E053
:101A0000F822E8C0E0786BE2F572D0E0F82275F0D9
:101A10000384B40104741A8017B402047422801081
:101A2000B40304742A8009B4040474428002741A52
:101A3000227403F97466F8752F0075308C7531E5E2
:101A4000120AB87866E2121A0E7869F27867E21222
:101A50001A0E786AF27868E2121A0E786BF2740144
:101A6000F97465F8752F0075308C7531E2120AB87B
:101A7000227403F97466F8752F0075308C7531E5A2
:101A8000120A017401F97465F8752F0075308C75B0
:101A900031E2120A01227976774809774E09777781
:101AA0000977A07404F97476F8752F0075308D7578
:101AB0003120120A327404F97476F8752F027530E9
:101AC0008D753120120A3222E4A21B92E0A21C92F0
:101AD000E1A21D92E27976F77401F97476F8752F18
:101AE0000075308C7531E8120A32227401F974766F
:101AF000F8752F0075308C7531E8120ADD7976E7BC
:101B0000A2E0921BA2E1921CA2E2921D227976E44D
:101B1000A22C92E0A22D92E1A22E92E2A21392E3D5
:101B200092E492E5A23092E6A23192E7F709E4A2AC
:101B30002F92E0A23292E1A23392E2A23492E3A287
:101B40003692E4A23692E5A23792E6A23892E7F7FF
:101B500009E4A23992E0A23A92E1A23B92E2A23CCD
:101B600092E3A23D92E4A23E92E5A23F92E7F709FA
:101B7000E4A24092E0A20192E1A20292E2A241928A
:101B8000E3A24392E4A24492E5A24592E6A24292E5
:101B9000E7F77404F97476F8752F0075308C753199
:101BA000EC120A327976E4A24692E1A24792E2A2CE
:101BB0004892E3F4F709E4F4F709E4F4F77403F95D
:101BC0007476F8752F0075308C7531E9120A32225F
:101BD0007404F97476F8752F0075308C7531EC1239
:101BE0000ADD7976E7A2E0922CA2E1922DA2E292A0
:101BF0002EA2E39213A2E69230A2E7923109E7A265
:101C0000E0922FA2E19232A2E29233A2E39234A2B6
:101C1000E4A2E59236A2E69237A2E7923809E7A25B
:101C2000E09239A2E1923AA2E2923BA2E3923CA274
:101C3000E4923DA2E5923EA2E6A2E7923F09E7A226
:101C4000E09240A2E19201A2E29202A2E39241A2BA
:101C5000E49243A2E59244A2E69245A2E79242743E
:101C600003F97476F8752F0075308C7531E9120A16
:101C7000DD7976E7F4A2E19246A2E29247A2E392EE
:101C80004809E7F409E7F4227976F77401F97476E4
:101C9000F8752F0075308C7531E4120A3222740108
:101CA000F97476F8752F0075308C7531E4120ADD01
:101CB0007976E7227401F9745BF8752F0075308C22
:101CC0007531FC120A01227401F9745BF8752F005A
:101CD00075308C7531FC120AB8227401F9745CF805
:101CE000752F0075308D753100120A01227401F9CB
:101CF000745CF8752F0075308D753100120AB822AA
:101D00007402F97472F8752F0075308C7531FD12FC
:101D10000AB87402F97474F8752F0075308D753136
:101D200001120AB8227402F97472F8752F00753026
:101D30008C7531FD120A017402F97474F8752F0064
:101D400075308D753101120A01227401F9745DF844
:101D5000752F0075308C7531F0120A017401F97419
:101D60005EF8752F0075308C7531F4120A0174011C
:101D7000F9745FF8752F0075308C7531F6120A0111
:101D80007401F97460F8752F0075308C7531F2129A
:101D90000A01227401F9745DF8752F0075308C7595
:101DA00031F0120AB87401F9745EF8752F007530BD
:101DB0008C7531F4120AB87401F9745FF8752F004C
:101DC00075308C7531F6120AB87401F97460F875C3
:101DD0002F0075308C7531F2120AB8227401F97433
:101DE00038F8752F0075308C7531F8120A3274018D
:101DF000F97439F8752F0075308C7531FA120A3282
:101E00007401F9743AF8752F0075308C7531FB1236
:101E10000A32227401F97438F8752F0075308C7508
:101E200031F8120ADD7401F97439F8752F00753034
:101E30008C7531FA120ADD7401F9743AF8752F00C5
:101E400075308C7531FB120ADD227402F9741EF8AC
:101E5000752F0075308C7531E0120A32227402F948
:101E6000741EF8752F0075308C7531E0120ADD2272
:101E7000C082C083E58275F008A42420F582500258
:101E800005F0A8F0E58375F008A4282400F5837810
:101E90007676FF7401F97476F8752F0085833085A6
:101EA0008231120A32A3A3A3A3A37401F97476F8B2
:101EB000752F00858330858231120A32D083D0821B
:101EC000C206220809E7C4F5F066540F700D08E752
:101ED000F5F066540F7004DAEAE422E6540FC5F018
:101EE000540FC395F09205740122787B79277A0309
:101EF000E6C4540FF309E6540FF30908DAF2792720
:101F0000789A7A06E6540FF6E36670080908DAF460
:101F1000E4C25322792C789F7A06C3E3961918DA23
:101F2000FA9205792C789F7A06E3540FB40F08E6ED
:101F3000540FB40F108008E6540FB40F0B8006182E
:101F400019DAE680CB740122C3E396B40902801249
:101F500014600FC3E3F5F0E695F0B40902800314B2
:101F600070E3E9B42704E4D253221918E366540F4E
:101F700060F080D1121EEA701A305317202F1575A9
:101F8000185085831985821A12178E7549B4D24F5D
:101F9000D252E42204227408F97476F8752F007581
:101FA000308C7531C0120ADD7498C395719571F843
:101FB000C3747B9571F9AA71121EC5227408F97455
:101FC00076F8752F0075308C7531C0120ADD121F3E
:101FD00074227405F97476F8752F0075308C75319C
:101FE000C0120A32227403F9747BF8752F00753021
:101FF0008C7531C5120A3222C082C083E58224204A
:10200000F582E583347DF5837401F9743BF8752F0F
:1020100000858330858231120ADDD083D082C08270
:10202000C083E58275F008A42420F582500205F0F3
:10203000A8F0E58375F008A4282400F5837408F956
:102040007476F8752F00858330858231120ADDD0D1
:1020500083D08222C082C083E58275F008A4242048
:10206000F582500205F0A8F0E58375F008A4282455
:1020700000F5837408F9748EF8752F008583308518
:102080008231120ADDD083D08222C082C083E582F1
:1020900075F008A42420F582500205F0A8F0E5832D
:1020A00075F008A4282400F5837406F97476F87591
:1020B0002F00858330858231120ADDD083D08222C1
:1020C0007405F97476F8752F00753000753120129B
:1020D0000ADD7498C395719571F8C3747B9571F995
:1020E000AA71121EC522751B20751C009000007479
:1020F00005F97476F8752F00851C30851B31120A9E
:10210000DD7498C395719571F8C3747B9571F9AAC4
:1021100071121EC56018E51B2408F51B5002051C32
:10212000A3E583B40FC9E582B4A0C4740122121FD1
:10213000F8E42220060280AE751B00751C0075684D
:102140009F75690FE568251BC2E0F582E569351CBE
:10215000F583C082C083E5822400F582E583341BC9
:10216000F5837402F97476F8752F018583308582C2
:1021700031120ADD78768683088682121FF87498F9
:10218000C395719571F8C3747B9571F9AA71121E8C
:10219000C57005D0F0D0F022D083D082C3E5831380
:1021A000F583E58213F582200514E58245836023DB
:1021B000E58224FFF568E58334FFF5698007A38590
:1021C000821B85831CC3E568951BE569951C40034C
:1021D000022144740122751B25751C0090000074B7
:1021E00003F9747BF8752F00851C30851B31120AAA
:1021F000DD121F746018E51B2408F51B5002051C36
:10220000A3E583B40FD9E582B4A0D4740122121FD0
:10221000F8E422789AE6540FB40F030222AD2006A8
:102220000280B3751B00751C0075689F75690FE50A
:1022300068251BC2E0F582E569351CF583C082C0C4
:1022400083E5822400F582E583343BF5837402F94B
:102250007476F8752F01858330858231120ADD7816
:10226000768683088682121FF8121F747005D0F0DC
:10227000D0F022D083D082C3E58313F583E58213A7
:10228000F582200514E58245836022E58224FFF56E
:1022900068E58334FFF5698007A385821B85831C6D
:1022A000C3E568951BE569951C4002808274012294
:1022B000788E7A0579A2E6540FC4F5F008E6540F3B
:1022C00045F0F70809DAEF22C2A3C260C2A2C263D6
:1022D000C2A1C262D2B775F002120652D5F0FA203E
:1022E000B72BD215D2A3C260C2A2D263D2A1C2625E
:1022F000D2A4C2611206ECB2B575F00F120652D527
:10230000F0FA30B7EF122384C2AF026F39D2A012B5
:102310000F70700712234812198A22C215754BFAE2
:1023200075F064120652D5F0FAC2A0C2A2C263755B
:10233000F064120652D5F0FAD2A0D2A2C263D2B78C
:1023400012066A30B79C80D3121AEB121BD0121CF3
:102350009EA2E09249A2E1924AA2E2924B121CC7CD
:10236000121CED121D93121E13121D00121E5D127F
:102370001A3122C2A3C260C2A2C263C2A1C262D287
:10238000A4C26122D2151260A140E8C2A3C260C2F9
:10239000A2C263C2A1C262D2A4C261C01EC01F7821
:1023A000769000007A08E6F008A3DAFA1224707832
:1023B000769000007A08E0F608A3DAFA900000129E
:1023C0005AB6121FD2121FE5D01FD01E121E4A127B
:1023D0005B301212D8120C6522751E30751F30C288
:1023E0001BC21CC21DC22CC22DC22EC213C230C2BF
:1023F00031C22FD232C233C234C236C237C238C21F
:1024000039C23AC23BC23CC23DC23EC23FC240C2D8
:1024100041C242C243C244C245C246C247C24878D2
:10242000727422F2087400F278747406F208740070
:10243000F2C249C24AC24B785B7404F2785C7409F8
:10244000F2785D7401F2785E7402F2785F7404F2DF
:1024500078607404F2753807753900753A007401B4
:102460007865F27866F2E408F208F2C207C2062242
:102470001210151223D9121E4A121AC8121B0DC2AD
:10248000E0A24992E0A24A92E1A24B92E2121C8899
:10249000121CB4121CDA121D4A121DDC121D251268
:1024A0001A71121A96126ABE22306504C26580093A
:1024B00075F00C20B205D5F0FAD322C322E8C0E0B3
:1024C000E9C0E0EAC0E07866E224FD40341224A9C5
:1024D00050257551007866E2600C75F003120652C3
:1024E000D5F0FA1238257865E2600C75F003120613
:1024F00052D5F0FA123999D0E0FAD0E0F9D0E0F8EC
:10250000223072F3C082C083E570700C12711F40DC
:1025100007122524D26BC26C1219EA1270F5D0830F
:10252000D08280D37866E275F00384E5F0B40007CA
:10253000124C47D25B801DB40107124BF3D25A8074
:1025400013B40210124B7E400B7859E583F208E574
:1025500082F2D25C22D25D8008C25D1225C7753C32
:1025600000C214D265754BFA7440301502740CF534
:1025700048C25BC24EE54860391224BD205B33750A
:10258000F003120652D5F0FA1207CF2015032014DB
:1025900018304EE1205D1B7548601217E5B40B0D35
:1025A00075F008120652D5F0FAD25B80051225BAF2
:1025B00080C3C25AD2AF754BFA22533C07F8E53CB0
:1025C000249AC8F6053C22789A75F00874FFF6083C
:1025D000D5F0FB22305A09201A03D21A22C25A22FD
:1025E000C21A22D25D8004D265C25DC214754BFA54
:1025F000D2197440301502740CF5481225C7753C89
:1026000000C25BC25AC24EC25CC25E1207CF201526
:102610000320142D1224BD205B29205A26205C2380
:10262000304E2A7865E27004C24E8021205D147518
:1026300048601217E5B40B1275F008120652D5F077
:10264000FAD25B754BFA126644221225BAE548604D
:10265000F2126644305EFD80B0E8C0E0785BE2F8DC
:10266000884C754D00B225E86002D225A225B392B0
:10267000A7D265D25FD0E0F82230140122789A7692
:102680000A0876038007789A760A0876010875F0BA
:102690006484F608E5F075F00A84F608A6F0753C47
:1026A00005D214227518C0751900751A0112178EFB
:1026B00022754700C2517518C0751900751A0212AB
:1026C000178E22D24F7549B475185075190F751AA7
:1026D000FF12178E22C209122659203B0C751810C2
:1026E00075190F751AFF12178E22203B0C751820D2
:1026F00075190F751AFF12178E2275186075190F4C
:10270000751AFF12178E2275187075190F751AFF3A
:1027100012178E22126ABE7518C0751900751A0E2E
:1027200012178E227876F208F2123BDB7518C0750C
:102730001900751A5012178E304300221228C1401A
:102740000D122AEE4008122CDF4003122E9F223079
:102750001508C37861E4F20228CCA290301B01B3C3
:102760007861E233F2B4FF0280060228CC02297BB2
:10277000201E032022F7D22230071CC0E078ACE2F2
:102780006013C3335005D0E002297B12069E50F639
:10279000D0E0022797D0E0785DE260D1B40128D282
:1027A0000A1226A430251720390C754D02754C02EB
:1027B000303D03754C01785CE2F54702297B2037F8
:1027C000031226C302297BB4021A12273C400F30A1
:1027D0002D03204D092067061226D502296D1226E9
:1027E000EA02297BB40308C24D1226FA02297BB4FF
:1027F0000705D271756F03B4090C204D032038030F
:102800000228B302297BB40A02743DB43408740070
:1028100012267902297BB435087410122679022910
:102820007BB43608741112267902297BB4370874F8
:102830002012267902297BB4381B7401F97476F8CA
:10284000752F0075308C7531F1120ADD7876E6123D
:10285000267902297BB4391B7401F97476F8752F37
:102860000075308C7531F1120ADD7876E612268615
:1028700002297BB43C0612271402296DB43D1320B3
:102880004D08D24D12270702296DC24D1226FA02B9
:10289000296DB43E0D304307E412272402296D024E
:1028A000297BB43F0E30430874FF12272402296DA0
:1028B00002297B751890751909F51A12178E0229CD
:1028C0007B785DE2B40B03A22222C32270F0201EAB
:1028D000033022EAC22230071CC0E078ACE2601369
:1028E000C3335005D0E002297B12069E50F6D0E09B
:1028F0000228F5D0E0785DE26022B40107C20A1236
:1029000026B18077B402028072B40307D24D122739
:10291000078068B40908204D46303843805DB40A0A
:1029200002743DB432028053B43302804EB4340298
:102930008049B435028044B43602803FB437028007
:102940003AB438028035B439028030B43C02802B6E
:10295000B43D028026B43E028021B43F02801C7543
:1029600018A0751909F51A12178E02297B10030396
:1029700002297B12669F120725D20322301508C355
:102980007862E4F2022AF9A291301C01B37862E283
:1029900033F2B4FF028006022AF9022BA8201E039C
:1029A0002023F7D22330071CC0E078ADE26013C3C8
:1029B000335005D0E0022BA812069E50F6D0E0025C
:1029C00029C4D0E0785EE260D1B40128D20A122690
:1029D000A430251720390C754D02754C02303D038B
:1029E000754C01785CE2F547022BA82037031226CC
:1029F000C3022BA8B4021A12273C400F302D03202B
:102A00004D092067061226D5022B9A1226EA022BC0
:102A1000A8B40308C24D1226FA022BA8B40705D2A7
:102A200071756F03B4090C204D03203803022AE0AE
:102A3000022BA8B40A02743DB4340874001226793B
:102A4000022BA8B435087410122679022BA8B436CC
:102A5000087411122679022BA8B4370874201226A4
:102A600079022BA8B4381B7401F97476F8752F001D
:102A700075308C7531F5120ADD7876E6122679020A
:102A80002BA8B4391B7401F97476F8752F007530D2
:102A90008C7531F5120ADD7876E6122686022BA8AF
:102AA000B43C06122714022B9AB43D13204D08D2D1
:102AB0004D122707022B9AC24D1226FA022B9AB406
:102AC0003E0D304307E4122724022B9A022BA8B4B0
:102AD0003F0E30430874FF122724022B9A022BA8C2
:102AE00075189075190AF51A12178E022BA8785EC0
:102AF000E2B40B03A22322C32270F0201E03302372
:102B0000EAC22330071CC0E078ADE26013C3335043
:102B100005D0E0022BA812069E50F6D0E0022B2230
:102B2000D0E0785EE26022B40107C20A1226B180CA
:102B300077B402028072B40307D24D12270780686F
:102B4000B40908204D46303843805DB40A02743D14
:102B5000B432028053B43302804EB434028049B49C
:102B600035028044B43602803FB43702803AB4382C
:102B7000028035B439028030B43C02802BB43D026F
:102B80008026B43E028021B43F02801C7518A075D7
:102B9000190AF51A12178E022BA8100303022BA88C
:102BA00012669F120725D2032230450E20460312DB
:102BB000274F20470312297C800612274F12297CB9
:102BC000301508C37863E4F2022CEAA292301D01AA
:102BD000B37863E233F2B4FF028006022CEA022DDE
:102BE00080201E032024F7D22430071CC0E078AEDA
:102BF000E26013C3335005D0E0022D8012069E50D0
:102C0000F6D0E0022C08D0E0785FE260D1B407058E
:102C1000D271756F03B4090C204D03203803022CC8
:102C2000D1022D80B40A02743DB434087400122617
:102C300079022D80B435087410122679022D80B4E3
:102C400036087411122679022D80B43708742012C8
:102C50002679022D80B4381B7401F97476F8752F2B
:102C60000075308C7531F7120ADD7876E612267918
:102C7000022D80B4391B7401F97476F8752F007534
:102C8000308C7531F7120ADD7876E6122686022D31
:102C900080B43C06122714022D72B43D13204D0857
:102CA000D24D122707022D72C24D1226FA022D7242
:102CB000B43E0D304307E4122724022D72022D800A
:102CC000B43F0E30430874FF122724022D72022DE8
:102CD0008075189075190CF51A12178E022D8078D0
:102CE0005FE2B40B03A22422C32270F0201E033043
:102CF00024EAC22430071CC0E078AEE26013C3337C
:102D00005005D0E0022D8012069E50F6D0E0022D34
:102D100013D0E0785FE26009B40908204D463038EE
:102D200043805DB40A02743DB432028053B433026E
:102D3000804EB434028049B435028044B4360280F7
:102D40003FB43702803AB438028035B4390280305B
:102D5000B43C02802BB43D028026B43E028021B4F4
:102D60003F02801C7518A075190CF51A12178E02F7
:102D70002D80100303022D8012669F120725D203B7
:102D8000301508C37864E4F2022EAAA28530280127
:102D9000B37864E233F2B4FF028006022EAA022F57
:102DA00059201E03202AF7D22A30071CC0E078B62B
:102DB000E26013C3335005D0E0022F5912069E5033
:102DC000F6D0E0022DC8D0E07860E260D1B407050B
:102DD000D271756F03B4090C204D03203803022E05
:102DE00091022F59B40A02743DB4340874001226BB
:102DF00079022F59B435087410122679022F59B46C
:102E000036087411122679022F59B437087420122B
:102E10002679022F59B4381B7401F97476F8752F8E
:102E20000075308C7531F3120ADD7876E61226795A
:102E3000022F59B4391B7401F97476F8752F007597
:102E4000308C7531F3120ADD7876E6122686022F71
:102E500059B43C06122714022F4BB43D13204D08E1
:102E6000D24D122707022F4BC24D1226FA022F4BCA
:102E7000B43E0D304307E4122724022F4B022F5992
:102E8000B43F0E30430874FF122724022F4B022F49
:102E90005975189075190DF51A12178E022F597859
:102EA00060E2B40B03A22A22C32270F0201E03307A
:102EB0002AEAC22A30071CC0E078B6E26013C333A6
:102EC0005005D0E0022F5912069E50F6D0E0022E97
:102ED000D3D0E07860E26022B40107C20A1226B1C2
:102EE0008077B402028072B40307D24D12270780A4
:102EF00068B40908204D46303843805DB40A027436
:102F00003DB432028053B43302804EB4340280495F
:102F1000B435028044B43602803FB43702803AB4FC
:102F200038028035B439028030B43C02802BB43D85
:102F3000028026B43E028021B43F02801C7518A096
:102F400075190DF51A12178E022F59100303022F4F
:102F50005912669F120725D203C21E20540122C2B5
:102F600054751840751900751A0012178E22E8C0A2
:102F7000E0785DE26403600A785EE264036003C3A4
:102F80008001D3D0E0F82212076F30070C12629054
:102F9000400390FFF11262D522C052122FB7D052D7
:102FA00022300713126290400390FFF11262D55055
:102FB00005F55212632C22E55270057552108023DC
:102FC000B41005755211801BB41105755220801381
:102FD000B420057552FF800BB4FF057552008003C5
:102FE0007552FF126393E55222C24D751860751930
:102FF0000F751AFA12178E22D24D75187075190FA7
:10300000751AFA12178E22C24D75186075190F7550
:103010001AE012178E22D24D75187075190F751A95
:10302000E012178E22E4A22592E0A22692E1A227C6
:1030300092E2A22B92E3F574757505123B5174036D
:103040005004123CD022123CAA7887E6C0E03046F9
:1030500012D0E0C0E0540712307DD0E0C0E0540749
:1030600012307D304714D0E0C0E0C454071232ABB8
:10307000D0E0C0E0C454071232ABD0E022A222302C
:103080001B01B34007D320E10A0232AAC320E203A6
:103090000232AA301B01B3301508C37861E4F20292
:1030A00031FB40060231FD0232AA201E032022F726
:1030B000D22230071CC0E078ACE26013C333500565
:1030C000D0E00232AA12069E50F6D0E00230D1D0F3
:1030D000E0785DE260D1B40128D20A1226A430253E
:1030E0001720390C754D02754C02303D03754C01AB
:1030F000785CE2F5470232AA2037031226C3023277
:10310000AAB4021A12273C400F302D03204D09208B
:1031100067061226D502329C1226EA0232AAB403AE
:1031200008C24D1226FA0232AAB40705D271756F91
:1031300003B4090C204D032038030231ED0232AAFA
:10314000B40A02743DB4340874001226790232AA1B
:10315000B4350874101226790232AAB436087411F4
:103160001226790232AAB437087420122679023264
:10317000AAB4381B7401F97476F8752F0075308C79
:103180007531F1120ADD7876E61226790232AAB498
:10319000391B7401F97476F8752F0075308C753110
:1031A000F1120ADD7876E61226860232AAB43C06CF
:1031B00012271402329CB43D13204D08D24D122721
:1031C0000702329CC24D1226FA02329CB43E0D30E8
:1031D0004307E412272402329C0232AAB43F0E3085
:1031E000430874FF12272402329C0232AA751890F9
:1031F000751909F51A12178E0232AA70FB201E03E8
:103200003022F5C22230071CC0E078ACE26013C364
:10321000335005D0E00232AA12069E50F6D0E002EA
:103220003224D0E0785DE26022B40107C20A12269F
:10323000B18077B402028072B40307D24D1227071F
:103240008068B40908204D46303843805DB40A02D6
:10325000743DB432028053B43302804EB4340280E1
:1032600049B435028044B43602803FB43702803A14
:10327000B438028035B439028030B43C02802BB4BB
:103280003D028026B43E028021B43F02801C7518A6
:10329000A0751909F51A12178E0232AA100303023B
:1032A00032AA12669F120725D20322A223301C01E4
:1032B000B34007D320E10A0234D8C320E20302342A
:1032C000D8301C01B3301508C37862E4F202342907
:1032D000400602342B0234D8201E032023F7D223C9
:1032E00030071CC0E078ADE26013C3335005D0E076
:1032F0000234D812069E50F6D0E00232FFD0E078B9
:103300005EE260D1B40128D20A1226A4302517202B
:10331000390C754D02754C02303D03754C01785CDB
:10332000E2F5470234D82037031226C30234D8B45A
:10333000021A12273C400F302D03204D092067064A
:103340001226D50234CA1226EA0234D8B40308C2BF
:103350004D1226FA0234D8B40705D271756F03B442
:10336000090C204D0320380302341B0234D8B40A60
:1033700002743DB4340874001226790234D8B4358E
:103380000874101226790234D8B436087411122643
:10339000790234D8B4370874201226790234D8B4AC
:1033A000381B7401F97476F8752F0075308C7531FF
:1033B000F5120ADD7876E61226790234D8B4391B84
:1033C0007401F97476F8752F0075308C7531F5122B
:1033D0000ADD7876E61226860234D8B43C06122737
:1033E000140234CAB43D13204D08D24D12270702EF
:1033F00034CAC24D1226FA0234CAB43E0D30430715
:10340000E41227240234CA0234D8B43F0E304308F1
:1034100074FF1227240234CA0234D8751890751923
:103420000AF51A12178E0234D870FB201E033023BF
:10343000F5C22330071CC0E078ADE26013C33350FF
:1034400005D0E00234D812069E50F6D0E002345285
:10345000D0E0785EE26022B40107C20A1226B18091
:1034600077B402028072B40307D24D122707806836
:10347000B40908204D46303843805DB40A02743DDB
:10348000B432028053B43302804EB434028049B463
:1034900035028044B43602803FB43702803AB438F3
:1034A000028035B439028030B43C02802BB43D0236
:1034B0008026B43E028021B43F02801C7518A0759E
:1034C000190AF51A12178E0234D81003030234D8E1
:1034D00012669F120725D203221235CF12366612CA
:1034E00036FD221235DC12367312370A22B20B3047
:1034F000071CC0E078B0E26013C3335005D0E0028F
:10350000355012069E50F6D0E002350ED0E0E53878
:10351000604C24F84005E538023569E538B4090403
:10352000A208803DB40A04A20A8036B40C03D380FA
:1035300030B40D0B3020030235E9D220D38022B401
:103540000E04A209801BB40F04A27180140235E995
:10355000B40D062020030235E9C220C38003A24D2A
:10356000B39226B392A50235E9300B60535003782D
:1035700050A2E2824F4030A2E082504012A2E1828B
:10358000514018C226A226B392A576000235E9B6AC
:103590000102801D7601754F408016B6020280112F
:1035A0007602754FA0800AB6030280057603754F38
:1035B000F0D25FE54F23F54F20E00AC226A226B3E2
:1035C00092A50235E9D226A226B392A50235E9E5F5
:1035D00038B40B07D226A226B392A522E538B40B45
:1035E00007C226A226B392A52230071CC0E078B1FC
:1035F000E26013C3335005D0E002364A12069E50F3
:10360000F6D0E0023608D0E0E539604C24F84005F9
:10361000E539023663E539B40904A208803DB40AED
:1036200004A20A8036B40C03D38030B40D0B3021D1
:1036300003023680D221D38022B40E04A209801B5B
:10364000B40F04A2718014023680B40D0620210349
:10365000023680C221C38003A24DB39227B392A643
:10366000023680023680E539B40B07D227A227B391
:1036700092A622E539B40B07C227A227B392A6224D
:1036800030071CC0E078B7E26013C3335005D0E0C8
:103690000236E112069E50F6D0E002369FD0E0E5F9
:1036A0003A604C24F84005E53A0236FAE53AB409A6
:1036B00004A208803DB40A04A20A8036B40C03D3E5
:1036C0008030B40D0B302903023717D229D3802262
:1036D000B40E04A209801BB40F04A2718014023737
:1036E00017B40D06202903023717C229C38003A28D
:1036F0004DB3922BB39280023717023717E53AB4D5
:103700000B07D22BA22BB3928022E53AB40B07C24F
:103710002BA22BB392802222B40207205B07C25A4D
:10372000C25C0237A6C082C08390EA60E53C606359
:1037300024FB405F789AE6540F758300F582D53CF0
:1037400002805075F00AA4F58275830008E6540FD4
:103750002582F582D53C02803AE58275F00AA4F50F
:103760008285F08308E62582F58250020583D53CE8
:10377000028020E58275F00AA4F582C0F0E5837529
:10378000F00AA4D0F025F0F58308E62582F58250F2
:103790000205837859E583F208E582F2C25BC25ADA
:1037A000D25CD083D08222C289C28BD293C2B4228F
:1037B000C0F075F0FAD5F0FD75F064D5F0FDD0F0ED
:1037C000221237B01237B01237B01237B01237B0FA
:1037D0001237B022D293C2B475F00512066A20B235
:1037E0000612066A30B203D5F0F112066A22C0F062
:1037F00075F008A2E7B392B4C2931237B0C2B4D244
:10380000931237B0C0E0E430B201040030B20104DA
:103810000030B20104D36003D5E001C3D0E033D55A
:10382000F0D1D0F022D293C2B4D2B21237B0C29348
:103830001237C1D2931237C1201503306C1C788621
:103840007601087480F608A2A3B392E4F674900897
:10385000F608F608F608F602389A788676030876AF
:1038600080087480A26092E5A2A3B392E4201508B8
:10387000A26392E1A22592E0F6087480201512203E
:103880006C0FE55154074480A26292E5A2A1B39265
:10389000E4F6087480F608F608F675F00778867E78
:1038A000007F00E62EFEE61237EEF62FFF08D5F079
:1038B000F2EED3331237EEF8EFD33368707A7886AE
:1038C000B6FF750561E56124FE501475610220178D
:1038D0000ED2177518C0751900751A0312178E20AD
:1038E00015087866E26003306C03023995788CE63F
:1038F00020E36C20E25C20E13D7887E6B6003708E3
:10390000B6421FD271756F037518B0751900751A1C
:103910000012178E7518C0751900751A0712178EC8
:103920008073B6551108B6000D087959E6F30809F9
:10393000E6F3D25CD26B805DE5616014D561113035
:10394000170EC2177518C0751900751A0412178E54
:1039500080437887863C08D25B799A7A04800B781A
:1039600087D25A757105798E7A05D26B75F00FE69C
:10397000C4540FF755F0F5F009E6540FF755F0F57C
:10398000F00908DAEAE5F0B40F051977EEC25A78C3
:1039900066E21237181237D422D293C2B4D2B212CE
:1039A00037B0C2931237C1D2931237C120151F30DE
:1039B0006B2378867611087480F608A2A3B392E48C
:1039C000F6749008F608F608F608F6023A1E7886AD
:1039D00076150239D978867613087680087480A225
:1039E0006092E5A2A3B392E4206B14A26192E1A2DB
:1039F000A4B392E0201508A26392E1A22592E0F61A
:103A0000087480206B0FE55154074480A26292E550
:103A1000A2A1B392E4F6087480F608F608F675F0F1
:103A20000778867E007F00E62EFEE61237EEF62F40
:103A3000FF08D5F0F2EED3331237EEF8EFD3336848
:103A4000706B7886B6FF660560E56024FE501475DD
:103A5000600220180ED2187518C0751900751A0565
:103A600012178E7865E26003306B03023B15788C89
:103A7000E620E36B20E25B20E14E7887E6B6002B80
:103A800008B64213D271756F037518C075190075A9
:103A90001A0712178E807EB6551108B6000D0879E8
:103AA00059E6F30809E6F3D25CD26C8068E5606001
:103AB00014D5601130180EC2187518C0751900752C
:103AC0001A0612178E023B15D26C7887863FD24EAB
:103AD00080437887863C08D25B799A7A04800B7899
:103AE00087D25A757105798E7A05D26C75F00FE61A
:103AF000C4540FF755F0F5F009E6540FF755F0F5FB
:103B0000F00908DAEAE5F0B40F051977EEC25A7841
:103B100065E21237181237D4227866E224FD40207D
:103B2000E2600C75F003120652D5F0FA12382578CF
:103B300065E2600C75F003120652D5F0FA1239995D
:103B400022306B0C7518B0751900751A0012178E9B
:103B500022D293C2B4D2B21237B0C2931237C1D2BA
:103B6000931237C17886E575540FC44407F608E50B
:103B70007423A2E392E5A2E292E3542AD2E7F60884
:103B8000E574A2E392E1A2E492E3542AD2E7F608B4
:103B9000E574A2E692E1A2E792E3540AD2E7F67452
:103BA0008008F608F608F675F00778867E007F0034
:103BB000E62EFEE61237EEF62FFF08D5F0F2EED332
:103BC000331237EEF8EFD33368700B7886B6FF0602
:103BD0001237D4C380041237D4D32275750878768F
:103BE000E2F574123B5174004005123CAA800312A6
:103BF0003CD07575097877E2F574123B5174014039
:103C000005123CAA8003123CD0227575047574FF1E
:103C1000123B5174025004123CD022123CAA788903
:103C20007954E6F30809E6F3087956E6F30809E65D
:103C3000F37887E6A2E092E25414F5F008E623A2B6
:103C4000E592E0540345F0F5F07858E265F0C0E005
:103C5000E5F0F2D0E030E21FC0E0C0F0E5F075F032
:103C60004930E20375F04A7518C075190085F01ADD
:103C700012178ED0F0D0E054037003023CA9E5F097
:103C80005403B4030575F0488013B4020575F0477A
:103C9000800BB4000575F04B800375F04C7518C0AF
:103CA00075190085F01A12178E22F5F0244AF8E2F1
:103CB000B40205227402F22250FA7402F2E5F024F2
:103CC00032F5F07518C075190085F01A12178E229A
:103CD000F5F0244AF8E26017D5E013F2E5F0243C51
:103CE000F5F07518C075190085F01A12178EF222BA
:103CF000D293C2B4D2B21237B0C2931237C1D293A8
:103D00001237C17886E575540FC44403F6087680EF
:103D1000087480A26092E5A2A3B392E4A26392E148
:103D2000A22592E0F6087480A26292E5A2A1B39265
:103D3000E4F6087480F608F608F675F00778867ED3
:103D4000007F00E62EFEE61237EEF62FFF08D5F0D4
:103D5000F2EED3331237EEF8EFD333687071788612
:103D6000B6FF6C788CE620E33020E22020E160781A
:103D700087E6B6005A08B6551108B60052087959B8
:103D8000E6F30809E6F3D25C804A80437887863CF4
:103D900008D25B799A7A04800B7887D25A757105BC
:103DA000798E7A0575F00FE6C4540FF755F0F5F0EB
:103DB00009E6540FF755F0F5F00908DAEAE5F0B432
:103DC0000F051977EEC25A786CE212371880051287
:103DD00037D4D3221237D4C322700575631E8002F4
:103DE000D21022C298C299322015F8309918C2997F
:103DF000205905753400800EC0E0C0D075D0101277
:103E000040E9D0D0D0E020980132C2982059FAC0C1
:103E1000D0C0E0E8C0E0305805C258754100E54523
:103E200024FE4003754502E54120E712E5415407B1
:103E30002324CFC0E07400343FC0E0E59922543F12
:103E4000232324C2C0E07400343EC0E0E59922156B
:103E500062023FC1023FC1D562FAB54408D20E7575
:103E60004100023FC7023FDFB462FA023FC1023F96
:103E7000C1B42AF1023FC1F56224C6E56240E624DE
:103E8000F5E56250E00562023FC17820F21562025A
:103E90003FC17821F21562023FC17822F215620219
:103EA0003FC17823F21562023FC17824F215620205
:103EB0003FC17825F21562023FC17826F2156202F1
:103EC0003FC1023FF500023E6800023E6E00023E26
:103ED0007100023E7700023E4F00023E4F00023E5C
:103EE0004F00023E4F00023E8A00023E9200023E18
:103EF0009A00023EA200023EAA00023EB200023E2A
:103F0000BA00023E5700023E5700023E5700023EF2
:103F10005700023E5700023E5700023E5700023E45
:103F20005700023E5700023E5700023E5700023E35
:103F30005700023E5700023E5700023E5700023E25
:103F40005700023E5700023E5700023E5700023E15
:103F50005700023E5700023E5700023E5700023E05
:103F60005700023E5700023E5700023E5700023EF5
:103F70005700023E5700023E5700023E5700023EE5
:103F80005700023E5700023E5700023E5700023ED5
:103F90005700023E5700023E5700023E5700023EC5
:103FA0005700023E5700023E5700023E5700023EB5
:103FB0005700023E5700023E5700023E5700023FA4
:103FC000F505412544F544D0E0F8D0E0D0D032806A
:103FD0000E802A802D8030803280348040803EB434
:103FE000090875440075410080D7B4420875440043
:103FF00075418080CC75440075410080CAB51EDFD4
:1040000080BFB51FDA80BAF54280B6F54380B2B5FD
:1040100044CD75452012401F75410080AA80D68589
:104020004236126DABD259E536B44603024E24B483
:104030004704126DC122B4500E854335126D86C2FD
:10404000ACC25975730722B45312854335E54370EA
:104050000A126D86C2ACC25975730222B4540E8521
:104060004335126D86C2ACC25975730122B4550E28
:10407000854335126D86C2ACC25975730322B4569E
:104080000E854335126D86C2ACC25975730422B4D5
:10409000570E854335126D86C2ACC2597573052221
:1040A000B4580E854335126D86C2ACC2597573067D
:1040B00022B44E21854335E543B4000B126D86C210
:1040C000ACC25975730822B4010B126D86C2ACC222
:1040D000597573092224BF24E6400485433522C262
:1040E0005922C5372537C53722E53424F0400EE57F
:1040F00034232408C0E074003441C0E022759906DE
:10410000C259753400D2B622802F80348036803870
:104110008039803E804680488051804F804D804B62
:1041200080468050800E0241B0753403F5991240EC
:10413000E2053422740002415E753700740380EC9E
:10414000E51E80E8E51F80E40241FEE53775340F87
:1041500080DA1217CC123DD9883580D0E53580C978
:10416000E535A24D92E080C1753403A8350535E6EA
:1041700076FF80B8E535C313603214700BA222922B
:10418000E0B392E1440480D614700BA22392E0B312
:1041900092E1440880C8147008A22492E0440C8084
:1041A000BD147008A22A92E0440C80B274FC80AE68
:1041B000E5351470107408A26692E0A26792E1A23D
:1041C0002592E280991470147410A22292E0A22326
:1041D00092E1A22492E2A22A92E3808214700D74EA
:1041E00018A21792E0A21892E102415E14700BA28D
:1041F0006892E0A26992E102415EE402415EE53626
:10420000B4410675340402412CB4422AE5356003FA
:1042100030101B53580F53590FC2AFE559B558060C
:10422000D2AFD302422E055953590FD2AFC3756393
:104230001E7442024129B444552007F7E535C313E3
:104240007022B39264122F6E404020303D30310B0B
:10425000204C05306434800320642FA264924D9278
:104260004C02428A926414C0E0030303540F247C7E
:10427000F8D0E0540704FA7400D333DAFD30640553
:10428000FAE24A8004F4FAE25AF6E53680A5B44B25
:10429000028003024323E53554F8B40812E535548F
:1042A00007603714604314604714605C0240FDB43B
:1042B000200FE5355407605914605C14605F0240BC
:1042C000FDB42813E535A2E0924D756E01500375DB
:1042D0006E02E5360241290240FD751AF4C267C23A
:1042E00066754C01754D01805E751AF3D26780EFDB
:1042F000751AF2D266C267754C01754D01C225A2CE
:1043000025B392A7D265803F751AF1D266C2678045
:1043100031C268C2698039D268C2698033C268D24A
:1043200069802DB4430FB5350375460375340775A1
:1043300035A202412CB44A20E53570192067167564
:104340001AF0C20912265975181075190F12178E16
:10435000E5360241290240FDB445067534060241A6
:104360002CB4510675340C02412CB44D0EE53512B7
:10437000182CE5365002B2E7024233B44C067534CD
:104380000E02412CB4460280C9B4470280C4B44F27
:1043900008C24FC250C25180B90240FDE565C26FEC
:1043A0006002D26FE552F553C252205C0C205A1BBA
:1043B000305B0302441B02492A12075D7859E2F57B
:1043C0008308E2F582121FF802452D12075D1222C2
:1043D000B0122133702820680820691F12499E50AE
:1043E0001AC082C08312072F122559D083D0823081
:1043F0005B0CE53C6008121F74700302452D754A82
:104400003CD5461475183075190085461A12178E5A
:10441000754603D2507549B402491512075DE53C53
:1044200060F6B40206125C6502492A206B1920145A
:1044300003303213B40510789AB60A0B08B601029D
:104440008008B6030280030244E608E675F00AA479
:10445000082675F00AA40826C5F0703B789BB603C1
:1044600039201409C0F0124959D0F0502A85F05271
:1044700085F05312072520140F7518C07519038590
:10448000521A12178E02492A7518C07519028552E0
:104490001A12178E02492A02490D201409C0F0127F
:1044A0004945D0F050F185F05220140E7518C075B2
:1044B000190685521A12178E800C7518C0751905C9
:1044C00085521A12178E12633012498BD2A2C26320
:1044D000C2A1D26212072F1225E7A25A725B5003C3
:1044E0000243AA02492A122213703F206808206959
:1044F0003C12499E503712072FC082C0831225E715
:10450000D083D082305A23C082C08312075D12222A
:10451000B0D083D0827498C395719571F8C3747BC1
:104520009571F9AA71121EC560030243FE306B3308
:1045300030071CC0E078B8E26013C3335005D0E008
:1045400002456312069E50F6D0E002454FD0E0755A
:1045500075027867E2786CF21219F6124C935003E8
:104560000243FE306C3330071CC0E078B9E26013C0
:10457000C3335005D0E002459912069E50F6D0E0B4
:10458000024585D0E07575037868E2786CF2121AFE
:1045900002124C9350030243FE7866E224FD500859
:1045A0001219EA1270F580031237A7E53B04700375
:1045B0000243FE754A00754603C251C250205202A2
:1045C000C24FC082C083124A45D083D082500612A7
:1045D00048C602492AC082C083120C7BD083D08295
:1045E00050061248C602492AE58224CEE58334FFEC
:1045F000501312498C400E122F6E50061248B7020B
:10460000492A02480712273C50121248B702479E17
:104610001248B102479E1248AB02479E2067F13014
:104620002D03204DF1E53B6058E53B600923120660
:104630009E400302463F0246811248A502479E3033
:1046400007F73013F4303EF1A26B303F01B3503125
:1046500030071BC0E078B5E26012C3335004D0E0ED
:1046600080D712069E50F7D0E002466ED0E0C0829E
:10467000C083126C2CD083D08250061248BC0247F3
:104680009E301349126BD8A2E09211A2E19212A2BD
:104690006B303F01B39204B40005200422802BB498
:1046A000012220041A7518C0751900751A0912170D
:1046B0008E203A061248C102479E12493B800E12D4
:1046C0006B558009B402ED2004DB126B7E30077954
:1046D00030071CC0E078B4E26013C3335005D0E06B
:1046E00002474912069E50F6D0E00246EFD0E02085
:1046F0006F16A26B926E85836685826712493712A8
:10470000074075650202492A756500E5836566F50F
:10471000F0E582656745F070061248CB02479E754A
:1047200018C0751900751A0C12178E306E0C75189A
:10473000B0751900751A0012178E1248F07518100E
:1047400085661985671A12178E304D0EC2A3C26096
:10475000C2A2C263D2A4C261800CD2A3C260C2A2B0
:10476000C263C2A4C261A26B9209D2081249331279
:10477000265930450620A803123025123B41124825
:10478000F075181085831985821A12178E12072565
:1047900030430BC082C083124B10D083D0821249A9
:1047A000955009124AC930E10302492A122F6E407E
:1047B000F8C2A1D262D2A4C261755100123B191293
:1047C0001FF8C082C0831225E7D083D082205C0905
:1047D000205A17205B2C02492A12075D7859E2B54E
:1047E000831D08E2B582180248077498C395719535
:1047F00071F8C3747B9571F9AA71121EC560080225
:104800004915121F7470F8301324E4A21192E0A22B
:104810001292E1B40305126BAA8013B40205126B65
:1048200055800BB40105126B7E8003126B2C300790
:104830001CC0E078B2E26013C3335005D0E00249F7
:104840001512069E50F6D0E002484DD0E030400FE1
:10485000E5824583600902485F12489F02492AB2F7
:104860004D123B41304D1A75187085831985821A97
:1048700012178EC2A3C260D2A1C262D2A4C261804A
:104880001875186085831985821A12178ED2A3C2F3
:1048900060D2A1C262C2A4C26112072502492A12D3
:1048A000663A0248CE12663A0248CE12663A02488A
:1048B000CE12663A0248CE12663A801212663A80EA
:1048C0000D12663A800812663A800312663A7565E0
:1048D000007566FF7567FF1234D9123B41751820C9
:1048E00085831985821A12178E1207121234E32259
:1048F000204803206B16E552046011146564600CB7
:104900007518C075190185521A12178E2212663A4F
:10491000120701801512663A1234D91207011234B7
:10492000E37565007566FF7567FFC25BC25AE553A4
:10493000F5522212663A2212663A2212663A75F04F
:1049400032120779227408F97476F8752F017530E0
:1049500003753198120ADD80127408F97476F875BF
:104960002F01753003753190120ADD787BE6085609
:10497000085604601412072F122559305B09E53CD4
:104980006005121F746002C322D32222E582249C98
:10499000E58334FF22E582249CE58334FF22A24A8A
:1049A000E58245836010E582249CE58334FF500452
:1049B000A2498002A24B22E5822582F582E5833559
:1049C00083F583E5822582F582E5833583F583E5EA
:1049D000822400F582E583345BF5837404F9740066
:1049E000F8752F01858330858231120AB822787BD1
:1049F000E654C0F583787CE630E402240A2323548D
:104A00003C4583F583787BE6C4540375F00AA4F52E
:104A1000F0E6540F25F0030303F5F053F0E085F0C2
:104A20008254034583F583787AE6C4540375F00A0B
:104A3000A4F5F0E6540F25F04582F58222C3958255
:104A4000E5F09583221249B77800E2B4FF03024AE9
:104A5000C51201621249EE7876A68308A682780014
:104A6000E2F58308E2F58208E2F5F008E2124A3D39
:104A7000502B7800E2F58308E2F582787686F0081C
:104A8000E6124A3D50417802E2F58308E2F5827869
:104A90007686F008E6124A3D402D024AC57800E2CB
:104AA000F58308E2F582787686F008E6124A3D4002
:104AB000167802E2F58308E2F582787686F008E659
:104AC000124A3D5002C322D322E5822418E58334E2
:104AD000FC74FFF5F05038C082C083C3E58233F523
:104AE00082E58333F583E5822400F582E583349AF9
:104AF000F5837402F97400F8752F0185833085827F
:104B000031120AB87801E2F5F018E2D083D082229F
:104B1000E5822400F582E58334BAF5837401F974E3
:104B200076F8752F01858330858231120ADD78761B
:104B3000E660422323C0E05403F5F0D0E054FC24A7
:104B400000F582E5F034CAF5837404F97476F875DB
:104B50002F01858330858231120ADD7876E608865A
:104B6000F07876F208E5F0F275F002120652D5F010
:104B7000FA123BDB2274FF7876F208F280EAE572E3
:104B8000B4220575F0048013B42A0575F006800B75
:104B9000B4420575F00C800375F0027836E2540FCC
:104BA000704F08D5F0F7E2540F75F00AA4F582753E
:104BB000830008E2540F2582F582E58275F00AA48D
:104BC000F58285F08308E22582F58250020583E5AF
:104BD0008275F00AA4F582C0F0E58375F00AA4D0CE
:104BE000F025F0F58308E22582F58250020583C3A3
:104BF00022D3227836E572B4220A75710479907551
:104C0000F0088024B42A0A757105798E75F00A803F
:104C100017B4420C757105798E75F00A783C8008DE
:104C2000757103799275F006E2F70809D5F0F9225B
:104C3000124BF37498C395719571F8C3747B957199
:104C4000F9AA71121EC522799A77000975F00577C5
:104C5000FF09D5F0FA75F008E572B42204783680C1
:104C600013B42A047838800CB44204783E80057866
:104C70003675F006753C06E2540F700608D5F0F75D
:104C80008009799AE2F70809D5F0F922124C471207
:104C90001F7422786CE27003024D3A24FD4048C034
:104CA00082C08312072F124D3ED083D082205C2613
:104CB000205B1B305A417498C395719571F8C37489
:104CC0007B9571F9AA71121EC5702C024D3A121F04
:104CD000747024024D3A7859E2B5831B08E2B5821C
:104CE00016658270128053C082C08312072F127122
:104CF000C1D083D0825003024D3C786CE275F00342
:104D000084E5F0B40007124C8C70EC802DB40107E0
:104D1000124C3070E28023B4021EC082C083124B5A
:104D20007EE5828583F0D083D08240CB658270C7D8
:104D3000E5F0658370C1800280BDC322D32275482F
:104D400032D265305E09C25EC0751207CFD075E5FC
:104D500048D36018C25CC25BC25A1224A950E41244
:104D60003CF0205C06205B03305AD8C3C0D0A87545
:104D70007405B802027404D0D04005123CAA800326
:104D8000123CD022C5372537C53722E54A24E940F1
:104D900008D2A3C260D2A2C2633098EFC298E5994C
:104DA000124D84223099FDC299F599124D8422C288
:104DB000A3C260C2A2C263C2B67537007405124DA9
:104DC000A4E51E124DA4E51F124DA4221206821264
:104DD0000682120682124DAFE536124DA4E5371257
:104DE0004DA43099FD22120FD4024DEF120F70C066
:104DF000E0124DAFE536124DA4D0E0124DA4E537D8
:104E0000124DA43099FD22120682124DAFE53612E2
:104E10004DA47976E7124DA409DDF9E537124DA4CA
:104E20003099FD22751A00754A19D215E538600BC4
:104E300054F87007C226A226B392A5E539600B5438
:104E4000F87007C227A227B392A6D2A0C28EC28C46
:104E5000C2ADC2ABC2ACC2AF7581C7904E66C08254
:104E6000C08375D00032D2AFD28C126D86C2ACD264
:104E700099124DCCB2B5754A19D298024EA3B40915
:104E800022F537124D8BB51E27124D8BB51F2112FF
:104E90004D8BB4461B124D8BAF37124D8B6F70107C
:104EA000124DCCD2B6D2A3C260D2A2C263124D8B35
:104EB000B40ACBF537124D8BB51EF5124D8BB51FCD
:104EC000EF124D8BF536B46D03024F53B46E0302EF
:104ED0004F6CB46F03024FA3B47003024FF0B47170
:104EE00003025004B47303025015B4740302501744
:104EF000B4750302502BB47603025043B477030217
:104F00005057B4780302506BB4790302508CB47AD2
:104F1000030250A8B46C030250BCB46B030250DE11
:104F2000B46A03025119B46903025135B46803022B
:104F30005194B467030251ACB466030251C7B4651F
:104F40000302528BB46403025A03B46103025A5E33
:104F5000024EA3AF37124D8B6F70F5124DCCD2B607
:104F600075F01E120652D5F0FA026F39124D8BFD04
:104F70001424E0402B124D8B2400FC7B00124D8B3F
:104F8000FEAF37124D8B6F70178EF0EDF97476F817
:104F90008B2F8C3085F031120ADD124E07754A19BD
:104FA000024EA3124D8BFD1454E070F4124D8B246D
:104FB00000FC247140EA7B02124D8BFEEDFA7876FC
:104FC000124D8BF608DAF9AF37124D8B6F70D1C2E4
:104FD000A3C260C2A2C2638EF0EDF97476F88B2F83
:104FE0008C3085F031120A32124DD5754A1980B0D5
:104FF000AF37124D8B6F70A8120D92124DCC754ABF
:1050000019024EA3AF37124D8B6F7009124DEC751C
:105010004A19024EA38089124D8BFD1424E04048AA
:10502000124D8B2400FC7B01024F7D124D8BFD1431
:1050300054E07034124D8B2400FC2425402A7B035D
:10504000024FB8AF37124D8B6F701D025068124D72
:10505000D5754A19024EA3AF37124D8B6F700912E6
:105060004DE6754A19024EA3024FA079207D071222
:105070004D8BF309DDFCAF37124D8B6F70EA126276
:105080000F40E5120143124DD5024EA3AF37124D2A
:105090008B6F70D4120162120682124DAFE5361288
:1050A0004DA412090C024EA3AF37124D8B6F7066E0
:1050B0001212D8124DCC754A19024EA3124D8BFE16
:1050C000124D8BFD124D8BFCAF37124D8B6F70461E
:1050D000120CF84041124DCC754A19024EA3124DE4
:1050E0008BFE124D8BFDAF37124D8B6F7028120C5B
:1050F000C9120682120682124DAFE536124DA4EE99
:10510000124DA4ED124DA4EC124DA4E537124DA49E
:105110003099FD024EA3024FA0AF37124D8B6F7036
:10512000F5120682120682124DAFE536124DA41218
:1051300016B3024EA3AF37124D8B6F70D9120F68A2
:1051400060027401C0E0120FCC60027402D0F0451E
:10515000F0700A120DDD121A961212D8E4C0E01295
:105160004DAFE536124DA4D0E0C0E0124DA4E537B6
:10517000124DA475F003120652D5F0FA124DAFE5A8
:1051800036124DA4D0E0124DA4E537124DA430994B
:10519000FD024EA3124D8BFD1454E07027124D8B6F
:1051A0002400FC2471401D7B00024FB8124D8BFD82
:1051B0001454E0700F124D8B2400FC242540057B15
:1051C00001024FB8024FA0AF37124D8B6F70F5122E
:1051D0000682120682124DAFE536124DA4740112FA
:1051E0004DA4744E124DA47477124DA47448124D00
:1051F000A47430124DA47400124DA4748D124DA4E9
:105200007420124DA474DA124DA47400124DA474CB
:105210000F124DA474A0124DA47480124DA47400FA
:10522000124DA47400124DA47420124DA4740012E7
:105230004DA47400124DA47400124DA47400124DBC
:10524000A47400124DA47400124DA47400124DA455
:105250007400124DA47400124DA47400124DA47475
:1052600000124DA47400124DA47400124DA47400D9
:10527000124DA47400124DA47400124DA4E537120F
:105280004DA43099FD024EA3024FA0124D8BF58321
:10529000124D8BF5822460E58334F040EB12557497
:1052A000124D8BFD1454E070DF7800124D8BF20824
:1052B000DDF9AF37124D8B6F70CE124DCC75F00506
:1052C000120652D5F0FA124DD5751A013007B930D1
:1052D00006B61255E81255CE125582121FF8788E76
:1052E00079007A0A75F00FE3540FF652F00809DAE4
:1052F000F643F0F0E5F004788E79767A05121EC553
:10530000600B1253A35006751A040252881255CE30
:10531000125582121FF8789A790A7A0675F00FE30F
:10532000540FF652F00809DAF643F0F0E5F004788D
:105330009A797B7A03121EC5600B12544150067590
:105340001A060252881255CE125631751A65024E4F
:10535000A3C0E07830E583F208E582F2D0E022C015
:10536000E07832E583F208E582F2D0E022C0E0780E
:1053700030E2F58308E2F582D0E022C0E07832E244
:10538000F58308E2F582D0E022E5822400F582E58B
:1053900083341BF58322E5822400F582E583343BC8
:1053A000F58322125582AB83AC82901B00C08379B7
:1053B00000752F0385833075310090005D1209E779
:1053C000120B581209E7120BB690005D7A80E0A329
:1053D000F5F0E0A36C7005E5F06B6017DAF0D083B0
:1053E0000583740024C0E58334C550C1740512548C
:1053F000F0D322D083EA2AF5F0E4C395F0F58212C7
:105400005351788E79007A0A75F00FE3540FF652F3
:10541000F00809DAF643F0F0E5F004600C122138E8
:10542000700A74061254F0D322122138E5822582C4
:10543000F582E5833583F58312538912535F025851
:1054400008125582AB83AC82903B00C08379007513
:105450002F0385833075310090005D1209E7120B30
:10546000581209E7120BB690005D7A80E0A3F5F0C0
:10547000E0A36C7005E5F06B6017DAF0D08305836C
:10548000740024C0E58334A550C174051254F0D3D0
:1054900022D083EA2AF5F0E4C395F0F58212535145
:1054A000789A790A7A0675F00FE3540FF652F008ED
:1054B00009DAF643F0F0E5F004601D122223701BB8
:1054C000AB83AC82125582EBB58306ECB58202C386
:1054D0002274041254F0D322122223E5822582F58D
:1054E00082E5833583F58312539612535F02580881
:1054F000F51A22C082C083E58312620ED083D08267
:10550000C082C083E58212620ED083D08222C08224
:10551000C0837F00E58224F0C0E0E58334D8C0E09A
:105520005007D083D0820F80EBD0E0D0E07F00E541
:10553000822418C0E0E58334FCC0E05007D083D05B
:10554000820F80EBD0E0D0E07F00E582249CC0E0B9
:10555000E58334FFC0E05007D083D0820F80EBD0CA
:10556000E0D0E0E58275F00A84C0F0F5F0D0F0D02C
:1055700083D08222C0E07834E583F208E582F2D05D
:10558000E022C0E07834E2F58308E2F582D0E02240
:10559000787BE612620E787CE612620E787DE61267
:1055A000620E789AE612620E789BE612620E789C82
:1055B000E612620E789DE612620E789EE612620E88
:1055C000789FE612620E1210662212106622740094
:1055D000124DA47400124DA47400124DA474001254
:1055E0004DA47400124DA42275831B75821B75F0A7
:1055F00040C0F0C082C083752F01858330753100B3
:105600001209E7120B58D083D082C082C083752F55
:10561000038582307531001209E7120C1ED083D049
:105620008205830582D0F0D5F0C77532FF7533FF50
:10563000227401F97418F8752F0075300075310067
:10564000120ADD7401F97419F8752F017530D975D6
:1056500031FF120ADDAC18125582E5822420F58252
:10566000E583347DF583C082C0837401F9743BF80F
:10567000752F00858330858231120ADDD083D08278
:105680007401F97410F8752F00858330858231120A
:105690000A017810E2F5F0E518253BC395F0F518FE
:1056A000125582E58275F008A42420F58250020587
:1056B000F0A8F0E58375F008A4282400F5837408A9
:1056C000F97476F8752F00858330858231120ADDF2
:1056D0007876E5187A082608DAFCF518788E7900CD
:1056E0007A0A75F00FE3540FF652F00809DAF64320
:1056F000F0F0E5F00412611D789A790A7A0675F0E7
:105700000FE3540FF652F00809DAF643F0F0E5F033
:10571000041261257408F97476F8752F00858330BA
:10572000858231120A327876E5187A08C39608DA4B
:10573000FBF518125582C3E58233F582E58333F514
:1057400083C3E58233F582E58333F583E582240064
:10575000F582E583245BF583C082C0837404F97409
:1057600076F8752F01858330858231120ADDD0836A
:10577000D0827404F97412F8752F01858330858204
:1057800031120A0178767912E5197A0426F5F0E3E8
:10579000C5F0C395F00809DAF3F5197401F9741826
:1057A000F8752F00753000753100120A327401F956
:1057B0007419F8752F017530D97531FF120A3275D9
:1057C000831B75821B75F040C0F0C082C083752FAB
:1057D000038583307531001209E7120B58D083D04E
:1057E00082C082C083752F01858230753100120915
:1057F000E7120C1ED083D08205830582D0F0D5F04D
:10580000C77532FF7533FF2212537BE5828583F023
:1058100012536DC39582C0E0E5F09583D0F045F05A
:105820007002C322500302592312537BC0E0C3E528
:105830008224FEF582E58334FFF583D0E012535FC6
:10584000E5828583F012536DB58207E5F0B58302DA
:10585000C32212536DAF8312537BEFB58310AE8218
:105860009000347876E0F6A308E0F60258867EFED3
:105870008F8305837402F97476F8752F038583305E
:10588000753100120ADD7900752F038F30753100F4
:1058900090005D1209E7120B581209E7120BB68F40
:1058A0008375820012536D7D00E5836F7002AD82B7
:1058B000ED245DF58275830050020583C3EE9D20C3
:1058C000E05A03FCC082C083A3A3E0FAA3E0FBD0AC
:1058D00083D082EAF0A3EBF0A3DCE9EE245DF5824D
:1058E000758300500205837876E6F0A308E6F07928
:1058F00000752F038F3075310090005D1209E7129B
:105900000C0A1209E7120C1E852F32853033125310
:105910007BEFB583030259F70F02585774081254EE
:10592000F0D32212536DAF8312537BEFB58310AEC9
:10593000829000347876E0F6A308E0F60259577EAC
:10594000008F8315837402F97476F8752F038583AD
:10595000307531FE120ADD7900752F038F307531F5
:105960000090005D1209E7120B581209E7120BB6FE
:1059700012536D7DFEE5836F7002AD82ED245DF5FF
:105980008275830050020583C3ED9E20E06B03FC0B
:10599000C0E0C3E58224FEF582E58334FFF583D0C1
:1059A000E0C082C083E0FAA3E0FBA3EAF0A3EBF03F
:1059B000D083D082DCDAEE245DF58275830050025C
:1059C00005837876E6F0A308E6F07900752F038F5B
:1059D0003075310090005D1209E7120C0A1209E7D8
:1059E000120C1E852F3285303312537BEFB58303A3
:1059F0000259F71F025928C32274091254F0D32206
:105A0000024FA0124D8BF583124D8BF582AF3712EA
:105A10004D8B6F70EBC01EC01F85831E85821F12C9
:105A20001E4A7401F97476F8752F007530007531CF
:105A300000120ADD7876E6C3951EC3951FD01FD0ED
:105A40001E251E251FF67401F97476F8752F007552
:105A50003000753100120A32124DCC024EA3124DA5
:105A60008BF583AF37124D8B6F709512068212063D
:105A700082120682124DAFE536124DA47400124D0B
:105A8000A4E51A124DA47400124DA47400124DA482
:105A90007400124DA47400124DA4E537124DA430C9
:105AA00099FD024EA3905AADC082C083327581C762
:105AB00075D000026F39C082C083E5822420F58250
:105AC000E583347DF5837401F9743BF8752F008507
:105AD0008330858231120A32D083D082C082C08363
:105AE000E58275F008A42420F582500205F0A8F0A4
:105AF000E58375F008A4282400F5837404F974760E
:105B0000F8752F00858330858231120A32A3A3A352
:105B1000A374762404F5F07404F9E5F0F8752F0009
:105B2000858330858231120A32D083D082C2062228
:105B3000120F70C0E07401F97476F8752F0075309B
:105B400000753100120ADD7876E6D0F0C395F0F6E4
:105B50007401F97476F8752F0075300075310012F4
:105B60000A3222120701C2AF80FE30071CC0E07863
:105B7000B2E26013C3335005D0E0025C0B12069E04
:105B800050F6D0E0025B89D0E0D2A3C260C2A1D2BD
:105B900062D2A4C26112072F1225E7205A06205BA9
:105BA00030025C0B12076F122133705F124995406F
:105BB0005A20680820695612499E505112072F1228
:105BC0002559305B46E53C6042121F74703D025C13
:105BD0000DE53C603612076F122213702E124995A4
:105BE000402920680820692512499E502012072F5D
:105BF0001225E7305A157498C395719571F8C374DE
:105C00007B9571F9AA71121EC56002D3223040182B
:105C1000E58245836012E53B60092312069E40033E
:105C2000025C26025C2880E3B24DC3123B41304D3A
:105C30001A75187085831985821A12178EC2A3C22D
:105C400060D2A1C262D2A4C2618018751860858337
:105C50001985821A12178ED2A3C260D2A1C262C263
:105C6000A4C261C322789AE6B40A1708E6B40545CF
:105C7000122F6E4009125B6A400412072522120798
:105C8000012275F00AA4F5F008E625F0B46326D2E7
:105C9000A3C260C2A2D263C2A1D262D2A4C261C0B6
:105CA000E012072F1225E7900000121FF8205A0972
:105CB000205B35D0E01207012212076F7498C3955C
:105CC000719571F8C3747B9571F9AA71121EC57034
:105CD000E2304A4412072F122559305BD612076F63
:105CE000121F7470CE025D1812076FE53C60C4127B
:105CF0001F7470BF304A2112072F1225E7305AB3A4
:105D000012076F7498C395719571F8C3747B957180
:105D1000F9AA71121EC5709B12072FD0E0B40B08B0
:105D2000125FB84024025E2DB40C08125FF94019CE
:105D3000025E2DB40D08126024400E025E2DB40EDA
:105D40000B1260334003025E3C025E29B40F28123E
:105D5000016212617B401DF824DC4018E8787AF675
:105D600012617B400FF824A0400AE87879F612010E
:105D700043025E2D025E29B410028003025DEE1222
:105D80000162122555204E06122555304EE6121797
:105D9000E5C0E0D0E0F824F640DAE8131354C07808
:105DA0007BF612617B40CD60CBF824ED40C6E878ED
:105DB0007CF612617B40346032F824CE402DE878C6
:105DC0007B46F6122555204E06122555304E1C12E4
:105DD00017E5C0E0D0E0F824F94010E8131313549D
:105DE000C0787C46F6120143025E2D025E29B41192
:105DF000151217FDB4010C1217FDB407061260420C
:105E0000025E2D025E29B41320202CF71225E72014
:105E10005B0B305AEE121F96700F025B63E53C601D
:105E200008121FBC7003025B6312070122125B3071
:105E30007518C0751900751A0A12178E12072522D7
:105E4000753B00787675F00876FF08D5F0FA22EFFA
:105E5000C0E0C2537893797B7A06EA30E004E60822
:105E60008002E6C4540FFFEA30E004E7098002E74D
:105E7000C4540FB40F10BF0F10EA6406600B205318
:105E80001ED0E0FFE422BF0F06D0E0FF7401222005
:105E900053F7F5F08F406F6002D253DABD80DFE533
:105EA000F0C395405002F4041460D6B408DB80D1EE
:105EB000788E79767A057401B6FF02800FB7FF02FB
:105EC000800AE66770060809DAF8E42274012212F3
:105ED0005EDAE58245837001D3228005D0E0025F5F
:105EE0002B1217FDC0E024F640F2D0E075F00AA4B2
:105EF000F5828005D0E0025F2B1217FDC0E024F68A
:105F000040F2D0E0258275F00AA4F58285F0838006
:105F100005D0E0025F2B1217FDC0E024F640F2D05E
:105F2000E02582F58250020583C322D322C082C0BD
:105F300083900000122054125EB0701AE5828583AF
:105F4000F0D083D082B5821FC5F0B5831AC082C05D
:105F500083F58385F082A3E583B40FD8E582B4A0EE
:105F6000D3D083D082C322D322C082C083900000CA
:105F7000122054125E4F701AE5828583F0D083D0D0
:105F800082B5821FC5F0B5831AC082C083F58385B0
:105F9000F082A3E583B40FD8E582B4A0D3D083D038
:105FA00082C322D3221225E7305A3112611D121FFB
:105FB000D2C3229000008008125ECF401F12072F2C
:105FC0001225E7305A1612076F121FF812611D12C0
:105FD0005F2D4008753B00125AB6C322D32212250A
:105FE00059305BF8E53C24FD24FC40F01261251299
:105FF0001FE5C3229000008008125ECF40DE12072A
:106000002F122559305BD5121FF8126125E53C602F
:106010000B24FD24FC40C5125F6940C0753B001293
:106020005AB6C322125ECF4008125E40125AB6C35F
:1060300022D322125ECF4008121FF8126091B322C1
:10604000D322C20690002874D8F974FFF8752F0186
:10605000858330858231120F2075830175F01E759E
:106060002F00858330753100C0F0C0831209E7121C
:106070000F00D0830583D0F0D5F0E4907D0074202C
:10608000F974FFF8752F01858330858231120F2056
:10609000227876E6080808080856B4FF02D322C31F
:1060A00022751E30751F30C26BC26C75F005C0F0D2
:1060B000D2A3C260C2A2D263D2A1C262D2A4C26180
:1060C000125E401225E7D0F0205A09205B06D5F079
:1060D000DD02611812613D403F120725787BE6B46E
:1060E000FF05C32275F005C0F01225E7D0F0205B54
:1060F00006D5F0F3026118E53CB4021C789AE62458
:10610000F6401508E624F6400F789AE62430F51E8E
:1061100008E62430F51FC322120701D322788E79B6
:10612000767A058006789A797B7A03E608540FC45C
:10613000F5F0E608540F45F0F709DAEF22205A315E
:10614000305B36E53C600624FD24FC402C126125C2
:1061500012072F75F005C0F01225E3D0F0205A1178
:10616000204E06D5F0F00261791217E5B40B0A80D3
:106170000312611D753B00C322D322122555204E08
:1061800006122555304E2B1217E5C0E0D0E0F8245A
:10619000F6401F122555204E06122555304E13127B
:1061A00017E5C0E0D0E0F5F024F64006E8C445F07D
:1061B000C322D3221261C475F064120652D5F0FADC
:1061C0001206D42275F03C120779C2A075F03C1279
:1061D0000779D2A075F014120779C2A075F03C12AD
:1061E0000779D2A075F014120779C2A075F01412C5
:1061F0000779D2A075F014120779C2A075F01412B5
:106200000779D2A02275F00A84C0F0D0F02222785B
:1062100025E254C07078E275F00A84C445F07878BD
:10622000F67824E254C07066E275F00A84C445F042
:106230007879F67823E254E07054E275F00A84C469
:1062400045F0787AF67822E2604454E07040E275D6
:10625000F00A84C445F0C0E07820E2030354C0D0C3
:10626000F045F0787BF67821E2602354F0701FE26D
:1062700075F00A84C445F0C0E07826E254F8700E48
:10628000E2C42354E0D0F045F0787CF6C322D32258
:1062900090000075F019C0F07402F97476F8752F4B
:1062A00001858330858231120ADD7877B6FF02805E
:1062B0000E18E552300705B4FF02E564666011E58B
:1062C000822410F58250020583D0F0D5F0C8C32295
:1062D000D0F0A3D32230074DE58224FFF582E58379
:1062E00034FFF58375F019E5822480E58334FE5090
:1062F00005900000800AE5822410F5825002058393
:10630000C0F07402F97476F8752F018583308582A8
:1063100031120ADD7877B6FF02800518E6B552071C
:10632000D0F0D5F0C2C322D0F0A3D3222202635B07
:10633000300EFAC20E12620F40F312014302635E86
:106340007822E21262057821E21262057823E212D5
:1063500062057824E2126205026382120162787B90
:10636000E6C45403E6540F787CE6C45401E6540FA7
:10637000787AE6C4540FE6540F7879E6C4540FE6F1
:10638000540F30070A126290500512632C800312DA
:10639000639322E552B4FF069004530263D2B40023
:1063A000069002930263D2B4100690029C0263D25C
:1063B000B411069002A50263D2B420069002AF0287
:1063C00063D2E55275F06484C0F0D0E012620590AB
:1063D00002DB2220130122758205126ABC600F7550
:1063E000F002120652D5F0FAD582EF126ABE747529
:1063F000787C12078A5015207014D270126ABE750C
:1064000018C0751900751A0D12178E22C27012016C
:106410006220330420342E22787AE6543FF5F07956
:1064200072E365F0701C09E3787966701520351108
:10643000D235126ABE7518C0751900751A0D12177B
:106440008E2230342A787AE6543FF5F07974E36589
:10645000F0701C09E37879667015203511D2351279
:106460006ABE7518C0751900751A0D12178E22C2F2
:106470003522C2AC1217CC6024F518881912134BC0
:1064800053580F53590FC2AFE559B55806D2AFD381
:1064900002649B055953590FD2AFC380D7D2AC22A7
:1064A0007E007F7490000075F000E49325F0F5F015
:1064B000A3C3E5829EE5839F40F0E5F0700122E5ED
:1064C000F0C0E0E58312620EE58212620ED0E012A7
:1064D000620EC2ADC2ACD2151206EC20B7FA75F04E
:1064E000C8120652D5F0FA30B7FD75F0C812065240
:1064F000D5F0FA126D862275F064120C3120E51287
:1065000030E30F2212066AB2B512066AB2B5D5F0B0
:10651000F322C2AFB2B512066AB2B512066AD5F05E
:10652000D9C2A075F032126504D2A075F03212659E
:1065300004C2A075F032126504D2A075F032126563
:106540000475F09612650480D82230073C740078F8
:106550008C12079940337F087E007478787C12078C
:106560008ACE13CE05E0DFF420160E7400789C125C
:1065700007995005EE655460108E548E527518C000
:1065800075190485521A12178E22C2AF751810752C
:10659000190FF51A12178ED2AF223007097401783D
:1065A0008C1207995001227477787C12078AE49242
:1065B000E0C0E07476787C12078AD0E033FE2016C3
:1065C0000E7401789C1207995005EE655560D78EC0
:1065D00055EE20E10630E02E02662330E017A26778
:1065E000726650C2C267C266754C01754D0174F87F
:1065F00012658A80B1D267C266754C01754D01740F
:10660000F712658A80A020669DD266C267754C012C
:10661000754D01C225A225B392A7D26574F6126505
:106620008A8083A225826640F8D266C267C20912B8
:10663000265974F512658A0265A6C082C083D0838C
:10664000D082222222C2A075F014120652D5F0FA8E
:10665000D2A075F014120652D5F0FA22C2A075F03D
:106660003C120652D5F0FAD2A075F014120652D59B
:10667000F0FA2212664512664512665C126645758E
:10668000F064120652D5F0FA2212665C12664512C8
:10669000664512664575F064120652D5F0FA22304E
:1066A0004D09C2A3C260D2A4C26122D2A3C260C2F9
:1066B000A4C2612230074930071CC0E078B3E26011
:1066C00013C3335005D0E00266EC12069E50F6D09C
:1066D000E00266D6D0E0D268201603206A22751840
:1066E000C0751900751A0F12178E8014C268201613
:1066F00003306A0C7518C0751900751A1012178EC0
:10670000A268926A22094300A00954009F0966000A
:106710009E0977009D0989009C099B009B09AD009B
:106720009A09BF009909D2009809E4009709F70077
:10673000960A0A00950A1D00940A3000930A430045
:10674000920A5700910A6B00900A7F008F0A93000B
:106750008E0AA7008D0ABB008C0AD1008B0AE700C5
:106760008A0AFE00890B1400880B2B00870B43005C
:10677000860B5C00850B7500840B8E00830BA700D5
:10678000820BC100810BDB00800BF6007F0C100038
:106790007E0C2B007D0C47007C0C64007B0C810080
:1067A0007A0C9E00790CBB00780CDB00770CFB00A8
:1067B000760D1B00750D3B00740D5B00730D7D00A5
:1067C000720D9F00710DC200700DE4006F0E070086
:1067D0006E0E2C006D0E51006C0E76006B0E9B0041
:1067E0006A0EC100690EE900680F1100670F3900D9
:1067F000660F6100650F8900640FB300630FDE0050
:10680000621009006110340060105F005F7F4290E9
:106810006705E493A3F5F0E493A3C3958BE5F095A6
:106820008D5015A3A3DFEBE58224FFF582E58334C9
:10683000FFF583E49314800BA3E493BF42059067B4
:10684000058010C0E0E58224F9F582E58334FFF588
:1068500083D0E02290006DE0A28733F02290006E9A
:106860007400F090006D7455F090006F74FFF0901C
:1068700000717405F09000707412F0D28122D286FB
:10688000A2A4C0D0D2A475F000D5F0FDD5F0FDC211
:106890008E53890F438910758B00758D00C28FC28E
:1068A000AFC2A4D28E208603308FFAC28E308F06FC
:1068B000758BFF758DFFD2AFD0D092A422F024FE4D
:1068C0004005308102C28122900071E0D5E0EE7473
:1068D00042F012687ED281E58B2499E58D34F24036
:1068E00014E58B24E1E58D34F3400EE58B24E0E5DF
:1068F0008D34FC400874158006741180027412FEF9
:10690000900070E06E6010EEF020020B7518C075FC
:1069100019008E1A12178E221268546036046033E2
:1069200090006FE020E010D2E0F090006EE0700484
:106930007405F022E4F02290006EE0602914F070FB
:10694000252001227518C0751900751A1412178EAA
:1069500002696690006FE030E00DC2E0F090006EDA
:10696000E070D1743CF02290006EE060F914F07099
:10697000F52001F27518C0751900751A1312178EDB
:1069800080E41268C812691822C2B612687E1268C2
:106990000D7537007403124DA4E51E124DA4E51FBA
:1069A000124DA4744E124DA4740C124DA474001216
:1069B0004DA4740A124DA4C082C083A3A3A3E49380
:1069C00075F064A4C0E0E5F0124DA4D0E0124DA42F
:1069D000A3A3A3A3E49375F064A4C0E0E5F0124D73
:1069E000A4D0E0124DA4D083D082E493124DA4A38E
:1069F000E493124DA4A3A3A3E493124DA4A3E493A0
:106A0000124DA4E58D124DA4E58B124DA4E537126D
:106A10004DA43099FD22C2B67537007403124DA4FF
:106A2000E51E124DA4E51F124DA4744E124DA47420
:106A300008124DA47401124DA47406124DA478548A
:106A4000E2F5F0E5F0124DA408E2F5F0E5F0124DA4
:106A5000A47856E2F5F0E5F0124DA408E2F5F0E571
:106A6000F0124DA4244AF8E27858E2547FF5F07809
:106A70004CE2C36001D3E5F092E7F5F0E5F0124D8A
:106A8000A475F000E5F0124DA4E537124DA430993D
:106A9000FD22120B28C2847454120B42E4120B0222
:106AA000120B15F5F06448255E33F55EE5F0255FC1
:106AB000B2E003F55FD9E9D284222222E422758371
:106AC000DD75F010752F03858330753100C083C0EC
:106AD000F01209E7120F00D0F0D0830583D5F0E45F
:106AE0007532FF7533FF126ABB22026B1DC082C074
:106AF00083758205C082126ABCD082601CC2A075F8
:106B0000F00F120652D5F0FAD2A075F00512065217
:106B1000D5F0FAD582DE126ABED083D082E5822417
:106B200000C0E0E58334DDF8D0E0C322126AEDC096
:106B300082C083F5828883787676007401F9747652
:106B4000F8752F03858330858231120A32D083D0C5
:106B500082126ABB22126AEDC082C083F5828883EA
:106B6000787676027401F97476F8752F0385833090
:106B7000858231120A32D083D082126ABB22126A15
:106B8000ED126AEDC082C083F58288837876760143
:106B90007401F97476F8752F03858330858231127C
:106BA0000A32D083D082126ABB22126AEDC082C040
:106BB00083F5828883787676037401F97476F875A4
:106BC0002F03858330858231120A32D083D082121E
:106BD0006ABB22126AEA8003126AEDC082C083F5A2
:106BE0008288837401F97476F8752F038583308564
:106BF0008231120ADD7876E6B40102800CB402021A
:106C00008007B4030280027400D083D08222120B6A
:106C100028C2847454120B42E4120B02120B15B4F6
:106C20000205755E018002D9F3D28422755E00757B
:106C300083DD75F00F752F03858330753100C083B8
:106C4000C0F01209E7120B581209E77900126C0E16
:106C5000D0F0D0830583E55E7026D5F0D8752F037C
:106C60008583307531001209E7120B581209E77954
:106C7000A0126C0E7532FF7533FFE55E7002D322F1
:106C8000C322C28C758A45758C5DD28CB2002000FF
:106C90000132C0D0C0E0C0F075D008D25E2015042B
:106CA000E54B6002B2B51217E4126D67051DE51DD4
:106CB00020E03E20E13B20153F206305A225B39252
:106CC000A2E51D30E2031234EDE51D541F7015D20C
:106CD0005FE4B54C2BB5474AB54959B56361B56F0B
:106CE00062B54A66E4B54B48B5486DB5456EB54EDC
:106CF00072D0F0D0E0D0D032E51D541F60E380F1B7
:106D0000303D0CE54D24C24003D54DC9754D3CD5F1
:106D10004CC3C2082066BEC225A225B392A7D26585
:106D200080B3D547B3C2087549B4D251D25480A8B4
:106D3000154B80B4D549A4C24FC250C251809C1596
:106D400063809BD56F9BC2718097D54A9775460328
:106D5000301503025AA580831548808FD5458FD200
:106D600058808B154E808AE51DA2E330600292A305
:106D700030630292A230620292A122C2B62059026E
:106D8000D2B6126D863275C800C2ADC2AC75CBFFEB
:106D900075CA9875CDFF75CC98759853C298C299ED
:106DA000D2ACC2BC75C8347599062275C800C2AC95
:106DB000C2AD75980075CC2B75CDEBD2AD75C804FE
:106DC0002275C800C2ACC2AD759800E58A242BF5C7
:106DD000CC540F658C24EBF5CDD2AD75C80422C21E
:106DE000A8C2AAC289C28BC2ACC2A9C2AB7580FFBD
:106DF0007590FF75A0FF758F01120C3ED215D2A0C1
:106E0000754C00754D00C225A225B392A7C226A2DB
:106E100026B392A5C227A227B392A6E4F53B787CBD
:106E200075F010F2D5F0FCC266C267C268C269751F
:106E30003D0F753F0F751D04C24EC24FC250C25167
:106E4000754901754A00C254D25E757300C235C2DD
:106E500017C218D258C259754510E4F541F542F5EC
:106E600043F534F5361223D9751E00751F80E4F5FD
:106E700047F550F54FF558F559F53EC222C223C2E9
:106E800024C22A74377861F27862F27863F2743738
:106E90007864F2D21E75460375480178A27A0576A9
:106EA000FF08DAFBC20E7820E47A07F208DAFCC2A7
:106EB0000F7552FF855254C210C207C206C2367502
:106EC000631E756500C26FC20CC20DC208C209C242
:106ED0000AC26BC26C75610075600075F00A784A71
:106EE000E4F208D5F0FB7954E4F309F37956F30999
:106EF000F37858E4F2121961754BFAB2B57532FFA6
:106F00007533FFD270756E00782F740AF2D20312B7
:106F1000685DC271756F0175721A758901758A3E57
:106F2000758C5DC2B9D2A9D28CD2B6126D86D2AFA1
:106F3000D293C2B4D2B2B2B522C21575510375F064
:106F400003120652D5F0FAC26BC26C123999755110
:106F50000375F003120652D5F0FAC26BC26C1238F8
:106F600025C2AF0200007866E224FD50061219EA3D
:106F70001270F522C2AF754BFAB2B512066AB2B5FD
:106F800012066AB2B5D2A07581C775D000126DDF46
:106F900012663A1264A0126ABE1222C8754BFA1227
:106FA0001249126F66755103123B19120739751891
:106FB00080751904751A7712178ED21630070F12C2
:106FC00010E112654A12659A1263D31266B4D2B701
:106FD000D2AFC215C21600000020B70912066A20FF
:106FE000B7030222E23007153036031210E13007F2
:106FF0000C12654A12659A1263D31266B4E5656095
:1070000003D5650E126982304403123C0A126330C4
:10701000800CD2A3C260C2A1D262D2A4C261E563D5
:107020007006303603126472C263D2A1C262126665
:107030009FC26BC26CD2657867E2600D24FD400987
:10704000757502123CF0126F667868E2600D24FDDF
:107050004009757503123CF0126F6630450620A892
:10706000031230251225E7205B08205A05205C0218
:10707000801A302E0930500612663A02708412438C
:107080009C126F66782FE215E0F27008782F741466
:10709000F2026FCE026FEE00207221C0D0C0E0E895
:1070A000C0E0C0F0E54E7003857270754E08D27571
:1070B00012716BD0F0D0E0F8D0E0D0D0C28932208D
:1070C0007221C0D0C0E0E8C0E0C0F0E54E7003859A
:1070D0007270754E08C27512716BD0F0D0E0F8D0A6
:1070E000E0D0D0C28B32C2A8C2AAC293C2B4C0E060
:1070F000120652D0E0C293C2B4C289C28BD2B2D2BD
:10710000B3C272754E00857270C2B8D288D2A8C25E
:10711000BAD28AD2AA22C2A8C2AAC289C28B22E546
:1071200072141475F00884F5F0C0F07836E230E09F
:1071300002B27330E102B27330E202B27330E302A2
:10714000B27308D5F0E7D0F0E230E002B27430E17B
:1071500002B27430E202B27430E302B27408D5F0C5
:10716000E7207305307402C322D322E570B572079D
:10717000A27592730271B5B40107A275927402717F
:10718000B5C3E572149570403275F004842436F866
:10719000E205F0D5F006A27592E38016D5F006A2BE
:1071A0007592E2800DD5F006A27592E18004A27579
:1071B00092E0540FF2D57002D27222857270D272B0
:1071C000227548321270E6305E05C25E1207CFE5C6
:1071D0004860113072F1E570700A12711612711F59
:1071E0004002C322127116D32200000000000000EA
:1071F000000000000000000000000000000000008F
:10720000000000000000000000000000000000007E
:10721000000000000000000000000000000000006E
:10722000000000000000000000000000000000005E
:10723000000000000000000000000000000000004E
:10724000000000000000000000000000000000003E
:10725000000000000000000000000000000000002E
:10726000000000000000000000000000000000001E
:10727000000000000000000000000000000000000E
:1072800000000000000000000000000000000000FE
:1072900000000000000000000000000000000000EE
:1072A00000000000000000000000000000000000DE
:1072B00000000000000000000000000000000000CE
:1072C00000000000000000000000000000000000BE
:1072D00000000000000000000000000000000000AE
:1072E000000000000000000000000000000000009E
:1072F000000000000000000000000000000000008E
:10730000000000000000000000000000000000007D
:10731000000000000000000000000000000000006D
:10732000000000000000000000000000000000005D
:10733000000000000000000000000000000000004D
:10734000000000000000000000000000000000003D
:10735000000000000000000000000000000000002D
:10736000000000000000000000000000000000001D
:10737000000000000000000000000000000000000D
:1073800000000000000000000000000000000000FD
:1073900000000000000000000000000000000000ED
:1073A00000000000000000000000000000000000DD
:1073B00000000000000000000000000000000000CD
:1073C000000000000000000000000000000050521B
:1073D000343032207665722E3131392E30204864B7
:1073E000773A482034303030752033312D30382D05
:1073F00030342031313A343920204352433D008B20
:00000001FF
:0300000306028072
